:182000004440A8003420EF0060042000E0ECB70020022000E1ECB7008C
:18201800A0002000E2ECB70000002000E3ECB70050042000D8ECB700D6
:18203000A0082000D9ECB70090002000DAECB70060042000DBECB70025
:1820480060022000DCECB700A0002000DDECB70000002000DEECB7009E
:1820600016080700E0002000E7EAB700A0002000BAAAB700600420005C
:1820780008A0B7003220EF00004025000800B4001000BA0008A0B70066
:182090000880BF0078AAB7004004200008A0B7003220EF0000402500AF
:1820A8000800B4001000BA0008A0B7000880BF00C6A9B700A00420000A
:1820C00008A0B7003220EF00004025000800B4001000BA0008A0B7001E
:1820D8000880BF009AA8B7008003200008A0B7003220EF000040250008
:1820F0000800B4001000BA0008A0B7004004200008A0B7003220EF00EF
:18210800004025000800B4001000BA0008A0B7000880BF00C6A9B70008
:18212000A003200008A0B7003220EF00004025000800B4001000BA0059
:1821380008A0B7000880BF0098A9B700C003200008A0B7003220EF006E
:18215000004025000800B4001000BA0008A0B7000880BF009AA9B700EC
:18216800E003200008A0B7003220EF00004025000800B4001000BA00D1
:1821800008A0B7000880BF009CA9B7000004200008A0B7003220EF00E1
:18219800004025000800B4001000BA0008A0B7000880BF009EA9B700A0
:1821B0002004200008A0B7003220EF00004025000800B4001000BA0048
:1821C80008A0B7000880BF0062AAB700E60AAF0003003700000020009D
:1821E000C2A9B700090037006000200008A0B7003220EF000040250000
:1821F8000800B4001000BA0008A0B7000880BF00C2A9B700E64AAF00A2
:1822100008003700E62AAF000300370000002000DEA9B70002003700E7
:1822280010002000DEA9B70005003700E62AAF000300370020002000BB
:18224000DEA9B700000037000636EF000836EF000A36EF0040442600E0
:18225800A6A0B70000A025005EA9B7002026200060A9B700E0AF2C000D
:1822700068A9B700A05A25006AA9B700002123006CA9B70040652700C9
:182288006EA9B70080A92B0070A9B700C0ED2F0072A9B700100020006E
:1822A000B0A9B70000002000B2A9B700E00020005CA9B70010002000F8
:1822B80074A9B7000000200082A9B7001000200084A9B700F0FF2F0006
:1822D00088A9B700F0FF2F0086A9B70090062000E4A9B700F0082000F8
:1822E800E6A9B7003220EF00804725001000BA0022AAB700A047250012
:182300001000BA0024AAB70000002000C209BD00010232000036EF0074
:182318000236EF000436EF00C169EF00C289BF007CAAB700BA69EF004B
:18233000BB69EF00C689BF00CEA4B700F00020009AAAB700E306070050
:182348009A2AED00FDFF3A00F442A900F462A900ECC2A9003000200011
:18236000B8E9B700000F2000CD42B600B9E9B700F0002000B849B600F9
:18237800B949B700CDE2B7006000200090A9B7009029ED00FEFF3A00E1
:18239000F442A8006000200090A9B7009029ED00FEFF3A00F442A9002B
:1823A800500020009AAAB700C80607009A2AED00FDFF3A00F442A90017
:1823C000F462A900ECC2A90030002000B8E9B700000F2000CD42B60013
:1823D800B9E9B700F0002000B849B600B949B700CDE2B700600020002E
:1823F00090A9B7009029ED00FEFF3A00F442A8006000200090A9B700BA
:182408009029ED00FEFF3A00F442A900500020009AAAB700AD060700DB
:182420009A2AED00FDFF3A005053200090A9B7009029ED00FEFF3A002D
:18243800F442A900F462A900ECC2A90030002000B8E9B700000F200080
:18245000CD42B600B9E9B700F0002000B849B600B949B700CDE2B70070
:182468006000200090A9B7009029ED00FEFF3A00F442A80060002000B1
:1824800090A9B7009029ED00FEFF3A00F442A900500020009AAAB7002D
:182498008E0607009A2AED00FDFF3A005053200090A9B7009029ED0051
:1824B000FEFF3A00F442A900F462A900ECC2A90020002000B8E9B70010
:1824C800000F2000CD42B600B9E9B700F0002000B849B600B949B7002F
:1824E000CDE2B7006000200090A9B7009029ED00FEFF3A00F442A80053
:1824F8006000200090A9B7009029ED00FEFF3A00F442A9005000200030
:182510009AAAB7006F0607009A2AED00FDFF3A005053200090A9B700A2
:182528009029ED00FEFF3A00F442A900F462A900ECC2A9000000200069
:18254000B8E9B700000F2000CD42B600B9E9B700F0002000B849B60017
:18255800B949B700CDE2B7006000200090A9B7009029ED00FEFF3A00FF
:18257000F442A8006000200090A9B7009029ED00FEFF3A00F442A90049
:18258800500020009AAAB700500607009A2AED00FDFF3A00F442A900AD
:1825A000F462A900ECC2A90080002000B8E9B700000F2000CD42B600E1
:1825B800B9E9B700F0002000B849B600B949B700CDE2B700600020004C
:1825D00090A9B7009029ED00FEFF3A00F442A8006000200090A9B700D8
:1825E8009029ED00FEFF3A00F442A900200320009AAAB700350607009F
:182600009A2AED00FDFF3A00F442A900F462A900ECC2A9002000200066
:18261800B8E9B700000F2000CD42B600B9E9B700F0002000B849B6003E
:18263000B949B700CDE2B7006000200090A9B7009029ED00FEFF3A0026
:18264800F442A8006000200090A9B7009029ED00FEFF3A00F442A90070
:18266000500020009AAAB7001A0607009A2AED00FDFF3A00F442A9000A
:18267800F462A900ECC2A90080002000B8E9B700000F2000CD42B60008
:18269000B9E9B700F0002000B849B600B949B700CDE2B7006000200073
:1826A80090A9B7009029ED00FEFF3A00F442A8006000200090A9B700FF
:1826C0009029ED00FEFF3A00F442A900200320009AAAB700FF050700FD
:1826D8009A2AED00FDFF3A00F442A900F462A900ECC2A90000002000AE
:1826F000B8E9B700000F2000CD42B600B9E9B700F0002000B849B60066
:18270800B949B700CDE2B7006000200090A9B7009029ED00FEFF3A004D
:18272000F442A8006000200090A9B7009029ED00FEFF3A00F442A90097
:18273800500020009AAAB700E40507009A2AED00FDFF3A00F442A90068
:18275000F462A900ECC2A90060002000B8E9B700000F2000CD42B6004F
:18276800B9E9B700F0002000B849B600B949B700CDE2B700600020009A
:1827800090A9B7009029ED00FEFF3A00F442A8006000200090A9B70026
:182798009029ED00FEFF3A00F442A900200320009AAAB700C90507005A
:1827B0009A2AED00FDFF3A00F442A900F462A900ECC2A90010002000C5
:1827C800B8E9B700000F2000CD42B600B9E9B700F0002000B849B6008D
:1827E000B949B700CDE2B7006000200090A9B7009029ED00FEFF3A0075
:1827F800F442A8006000200090A9B7009029ED00FEFF3A00F442A900BF
:18281000500020009AAAB700AE0507009A2AED00FDFF3A00F442A900C5
:18282800F462A900ECC2A900C0002000B8E9B700000F2000CD42B60016
:18284000B9E9B700F0002000B849B600B949B700CDE2B70060002000C1
:1828580090A9B7009029ED00FEFF3A00F442A8006000200090A9B7004D
:182870009029ED00FEFF3A00F442A900200320009AAAB70093050700B7
:182888009A2AED00FDFF3A00F442A900F462A900ECC2A90000002000FC
:1828A000B8E9B700000F2000CD42B600B9E9B700F0002000B849B600B4
:1828B800B949B700CDE2B7006000200090A9B7009029ED00FEFF3A009C
:1828D000F442A8006000200090A9B7009029ED00FEFF3A00F442A900E6
:1828E800500020009AAAB700780507009A2AED00FDFF3A00F442A90023
:18290000F462A900ECC2A900F0002000B8E9B700000F2000CD42B6000D
:18291800B9E9B700F0002000B849B600B949B700CDE2B70060002000E8
:1829300090A9B7009029ED00FEFF3A00F442A8006000200090A9B70074
:182948009029ED00FEFF3A00F442A900200320009AAAB7005D05070014
:182960009A2AED00FDFF3A00F442A900F462A900ECC2A9000000200023
:18297800B8E9B700000F2000CD42B600B9E9B700F0002000B849B600DB
:18299000B949B700CDE2B7006000200090A9B7009029ED00FEFF3A00C3
:1829A800F442A8006000200090A9B7009029ED00FEFF3A00F442A9000D
:1829C000500020009AAAB700420507009A2AED00FDFF3A00F442A90080
:1829D800F462A900ECC2A90010002000B8E9B700000F2000CD42B60015
:1829F000B9E9B700F0002000B849B600B949B700CDE2B7006000200010
:182A080090A9B7009029ED00FEFF3A00F442A8006000200090A9B7009B
:182A20009029ED00FEFF3A00F442A900200320009AAAB7002705070071
:182A38009A2AED00FDFF3A00F442A900F462A900ECC2A900000020004A
:182A5000B8E9B700000F2000CD42B600B9E9B700F0002000B849B60002
:182A6800B949B700CDE2B7006000200090A9B7009029ED00FEFF3A00EA
:182A8000F442A8006000200090A9B7009029ED00FEFF3A00F442A90034
:182A9800500020009AAAB7000C0507009A2AED00FDFF3A00F442A900DD
:182AB000F462A900ECC2A90020002000B8E9B700000F2000CD42B6002C
:182AC800B9E9B700F0002000B849B600B949B700CDE2B7006000200037
:182AE00090A9B7009029ED00FEFF3A00F442A8006000200090A9B700C3
:182AF8009029ED00FEFF3A00F442A900200320009AAAB700F1040700D0
:182B10009A2AED00FDFF3A00E60AAE000B0037000000200000A4B7006B
:182B28000224EF0080FF2F0004A4B700CE24EF0000082000C0A4B7004F
:182B400000C02400C2A4B70001E4A800100020009AAAB700DF040700DA
:182B58009A2AED00FDFF3A002682BF002202AF00F8FF37002682BF00AF
:182B70002202AF00FDFF3700B42AEF00B22AEF00C86AEF00C76AEF006E
:182B8800C66AEF00B7EAEF0083E0A8002222A9002242A9008560A900F3
:182BA0009560A8008760A9008780A9009780A800A00020009AAAB700C6
:182BB800C60407009A2AED00FDFF3A000060FE0040A7A80093EAA9003A
:182BD000200320009AAAB700BE0407009A2AED00FDFF3A002062AE00CF
:182BE800030037000000200010A1B70011E1A8000000280012A1B700E7
:182C0000001920000EA1B7004087AE00010037001AAAEF003220EF007C
:182C180000C0B300ECEAB70060EDB70061EDB7006AEDB70066EDB70083
:182C3000CCEAB700FAEAB70010002000F9EAB70020002000F8EAB700E1
:182C480030002000F7EAB70040002000F5EAB70080002000F4EAB70061
:182C6000F0CFB300F3EAB700B7EAB700800220006BEDB700800F20009E
:182C7800F2EAB70010002000F1EAB700B0002000F0EAB700000C200062
:182C9000D3EAB70080002000DDEAB700B0002000DCEAB700000020002D
:182CA800E4EAB70000002000E5EAB70000002000E0EAB7000000200028
:182CC000E1EAB700C0FE2000EAAAB7002882BF000020EC002062AF00AB
:182CD800020037004100DD00010037004200DD0064AAB7000020EF0062
:182CF0006BCDBF00BA0AB400640ABC000680BF0003003A000480BF006E
:182D08000CA1B700010037000CA1EF00803E20002AAAB7002C2AEC00D0
:182D200061CDBF0001003A00EC02A90000E0200014A0B700CB6AEF004D
:182D38008C6AEF00E96AEF00A5040700ECCABF0088EAB70010C0B3008B
:182D5000B84AB50003003A0000CCB300EC4AB600060037000020EF00C0
:182D6800C9CABF0003003200C96AEF0000CCB300EC4AB600EEFF320020
:182D8000CBEAEF00F0C1B300884AB600D2EAB70000CCB300884AB60031
:182D9800D3EAB70000CCB300D34AB50004003A00F0CFB300884AB50027
:182DB00001003A00DDFF370000C8B300D34AB50027003A00D0CBB300C1
:182DC800884AB5000E003A0030C0B300664DB500050031000020EF00D4
:182DE00066CDBF000020B40016A0B700010037000B002000C4E9EF00A9
:182DF8008E89BF001620B4000B00900000400100F0C3B300884AB60039
:182E1000D1EAB700E9EAEF00D1CABF004200A90000C0D60000C0D60005
:182E280000C0D60000C0D60017E0B70000C0D700F24AB60016E0B70082
:182E400017C0BF00F14AB600F04AB40017E0B700C4E9EF003B407800C8
:182E580088EAB7000000370088CABF00005D780000CCB300884AB60015
:182E7000D3EAB700F0C3B300884AB600D1EAB70080C0B300884AB600FB
:182E8800CEEAB70040C0B300884AB600EEEAB70030C0B300884AB600CE
:182EA000EDEAB70000C2B300884AB600EFEAB70000CCB300D34AB500AE
:182EB8000A003A0000C2B300EF4AB50007003A0000C0B300E94AB500BF
:182ED000030032000B409000005D7800010037007204070000C4B300D9
:182EE800D34AB50065003A0040C0B300EE4AB5000A003A0000C0B3000A
:182F0000E94AB500050032003B407800005D78003B407800005D78000A
:182F180002003700630407006204070000C2B300EF4AB50055003A009B
:182F300000C0B300ED4AB5000A003A0000C1B300884AB60006003200B2
:182F480000C0B300E94AB500020032003B407800005D780001003700E2
:182F60005204070010C0B300ED4AB5000D003A0000C1B300884AB6004A
:182F78000800320000C0B300E94AB500040032003B407800005D7800AE
:182F90003B407800005D780002003700430407004204070020C0B300FA
:182FA800ED4AB50013003A0000C1B300884AB6000C00320000C0B3002B
:182FC000E94AB500080032003B407800005D78003B407800005D780047
:182FD8003B407800005D78003B407800005D7800040037002F040700DC
:182FF0002E0407002D0407002C04070030C0B300ED4AB5001F003A0039
:1830080000C1B300884AB6001400320000C0B300E94AB50010003200D1
:183020003B407800005D78003B407800005D78003B407800005D780040
:183038003B407800005D78003B407800005D78003B407800005D780028
:183050003B407800005D78003B407800005D780008003700110407007D
:18306800100407000F0407000E0407000D0407000C0407000B040700BD
:183080000A04070000C0B300E94AB50002003A0000C0B30088EAB700F0
:1830980000C0B3000045980000C0B300E94AB5000A0032003B40780046
:1830B00088EAB700005D780014C0BF00EA4AB50015C0BF00EBCAB50090
:1830C8000200310000C1B300616DB70088CABF0063FF3A00E96AEF00D5
:1830E00000C0B3000045980062CDBF00090032008CCABF0093030700AD
:1830F800ECCABF008C4AB5000400320010C0B300616DB700636DEC00C6
:1831100006FF3700CB6AEF0000E0200014A0B7008B6AEF003A40780006
:1831280088EAB70000CCB300884AB600D3EAB70080C0B300884AB60070
:18314000CEEAB70040C0B300884AB600EEEAB70030C0B300884AB60013
:18315800EDEAB70000C2B300884AB600EFEAB70000CCB300D34AB500F3
:18317000F0003A00F0C1B300884AB600D2EAB70000C2B300884AB600C1
:18318800EFEAB70016C0BF00E2EAB70017C0BF00E3EAB70000C1B300F9
:1831A000D24AB5002A00310000D6200016A0B70016C0BF00D24AB40023
:1831B80016E0B70017C0BF00FACAB40017E0B70000C2B300EF4AB50033
:1831D0001C003A003A40780080459800B0CEB300884AB50012003A003E
:1831E8002882BF000020EC002062AF00020037004100DD00010037009A
:183200004200DD0064AAB7000020EF006BCDBF00BA0AB400640ABC002A
:183218000680BF0003003A000480BF000CA1B700010037000CA1EF00A1
:1832300060CEB300884AB50001003A009F030700020037000B40900026
:183248008E030700B500370000C2B300EF4AB50042003A0070CFB30019
:18326000884AB50002003A003A4078003C00370080CFB300884AB500A5
:1832780009003A0000C0B3006A4DB50003003A003A407800E4EAB70068
:18329000020037003A407800E0EAB7003000370090CFB300884AB5007A
:1832A80009003A0000C0B3006A4DB50003003A003A407800E5EAB70037
:1832C000020037003A407800E1EAB70024003700A0CFB300884AB50045
:1832D80011003A0000C0B3006A4DB50007003A003A407800E44AB4009F
:1832F000E4EAB700E5CABF00FACAB400E5EAB700060037003A407800A6
:18330800E04AB400E0EAB700E1CABF00FACAB400E1EAB70010003700A3
:18332000D0CFB300884AB50003003A003A407800CCEAB7000A003700DF
:18333800E0CFB300884AB50007003A003A407800ECEAB700A0C5B300BC
:18335000EC4AB50001003A0029FB3700000037007000370000CDB30086
:18336800884AB50003003A0070C3B300430307006A00370010CDB30025
:18338000884AB50003003A0090C4B3003D0307006400370020CDB300E8
:18339800884AB50003003A0070C3B300370307005E00370030CDB300ED
:1833B000884AB50003003A0030C3B300310307005800370040CDB30011
:1833C800884AB50003003A00D0C0B3002B0307005200370050CDB30058
:1833E000884AB50003003A00E7CABF00250307004C00370060CDB3000F
:1833F800884AB50003003A00E6CABF001F0307004600370070CDB300F4
:18341000884AB50003003A0040C9BF001903070040003700A0CDB3005E
:18342800884AB50003003A0000C0B300130307003A003700B0CDB30097
:18344000884AB50003003A007BCDBF000D03070034003700D0CDB300D7
:18345800884AB50003003A0000C0B300070307002E003700E0CDB3004F
:18347000884AB50003003A0020C0B3000103070028003700C0CDB30043
:18348800884AB50003003A0080C0B300FB02070022003700C0CDB300D8
:1834A000884AB50003003A0080C0B300F50207001C00370080CDB3000C
:1834B800884AB50008003A0000C0B3006A4DB50002003A00E4CABF00AB
:1834D00001003700E0CABF00EA0207001100370090CDB300884AB50071
:1834E80008003A0000C0B3006A4DB50002003A00E5CABF0001003700C9
:18350000E1CABF00DF02070006003700F0CDB300884AB50003003A00F0
:18351800A0C5B300D902070000003700E2CABF0016E0B700E3CABF00E6
:1835300017E0B700F0C3B300884AB600D1EAB70000C4B300D34AB5002C
:18354800E0013A0040C0B300EE4AB5000C003A0000C0B3006A4DB5008B
:1835600005003A003A407800E4EAB7003A407800E5EAB70004003700EA
:183578003A407800E0EAB7003A407800E1EAB70000C0B3006A4DB50075
:1835900005003A00E4CABF0016E0B700E5CABF0017E0B7000500370072
:1835A800E0CABF0016E0B700E1CABF00F04AB40017E0B70020C0B3005C
:1835C0006C4DB50002003A004200A9000600370000C0B3006A4DB50042
:1835D80002003A004200A900010037004200A9000400390000DB200059
:1835F00016A0B70000C2B300616DB70010C0B3006C4DB50016003A001B
:183608003220EF004200F800000E20004200B70042A0B70000DB200074
:183620001AA0B70000402500E44AB40018A0B70080002000ACAAB700BE
:183638001880BF001040BA00804698001820EC001A20EC00AC2AED00AE
:18365000F9FF3A0000DB200016A0B7004200F90020C0B3006C4DB5008C
:1836680034003A0080002000DDEAB700B0002000DCEAB7004200A90086
:18368000DA8ABF000080D700D6AAB700D88ABF000080D7000000A90060
:18369800D4AAB700F0FF2700E40AB6004200A9000080D7000000A90040
:1836B000D40AB400D4AAB70000C8B300E54AB6001B003A0000DB20008B
:1836C80016A0B70000C2B300EF4AB500150032001400F800D68ABF00A8
:1836E00032A0B700D48ABF0014A0B70000DB20001AA0B7001480BF0002
:1836F8001000BA00801E78001480BF001080BA00801E780014A0EC0087
:183710001480BF001000BA00801E78001480BF001080BA00801E7800BB
:183728001400F9000300370080AD2000E44AB40016A0B70000C2B30031
:18374000EF4AB500FB003A0000C0B300ED4AB50004003A003A407800BF
:18375800805D7800F9CABF00E101070010C0B300ED4AB50007003A00E9
:183770000400FC003A407800805D78003A407800805D7800F8CABF0032
:18378800D701070020C0B300ED4AB5000B003A000800FC003A40780090
:1837A000805D78003A407800805D78003A407800805D78003A4078003C
:1837B800805D7800F5CABF00C901070030C0B300ED4AB50013003A0079
:1837D0001000FC003A407800805D78003A407800805D78003A40780055
:1837E800805D78003A407800805D78003A407800805D78003A407800F4
:18380000805D78003A407800805D78003A407800805D7800F4CABF0050
:18381800B30107003A11070010C0B3006C4DB50052003A003220EF00CD
:183830004200F800000E20004200B70042A0B700E5CABF0047003A0097
:1838480000C8B300E44AB60040003A001400F8000040250014A0B700B3
:1838600000042000ACAAB7001480BF001000BA00000DBB00000020001A
:18387800008DBB0014A0EC00AC2AED00F8FF3A003220EF0020042400D3
:1838900060A7B7000040250014A0B7001000BA00000DBB0040A7A90070
:1838A8004200F800000E20004200B70042A0B7005005200066A7B700D5
:1838C000A00A200066A7B70061E7A80000000000000000004200F90037
:1838D8000060FE0000DB20001AA0B70000402500E40AB40014A0B7009C
:1838F00080002000ACAAB7000D409000004DBB001420EC001A20EC00E8
:18390800AC2AED00FAFF3A0040A7A9001000240060A7B70050052000BA
:1839200066A7B700A00A200066A7B70061E7A80000000000000000004D
:1839380061E7AF00FEFF37000000200060A7B7000060FE001400F90003
:183950000300370000C2B300616DB7006C6DEF000300370000C2B300B4
:18396800616DB7006C6DEF004200F90020C0B3006C4DB5006C003A0018
:1839800070C7B300DF4AB50014003A004200F800000E20004200B700B8
:1839980042A0B7001400F800D68ABF0032A0B700D48ABF0014A0B70042
:1839B000000420000AA0B700F0FF2F00000DBB00008DBB0014A0EC00AC
:1839C8000A20ED00FAFF3A001400F900DF6AEF004200F900D0CFB300CB
:1839E000DF4AB50017003A004200F800000E20004200B70042A0B700A6
:1839F8001400F80040A7A9001000240060A7B7005005200066A7B700F0
:183A1000A00A200066A7B70061E7A800000000000000000061E7AF0029
:183A2800FEFF37000000200060A7B7000060FE001400F900DF6AEF00D1
:183A40004200F900E0CFB300DF4AB5001D003A004200F800000E200034
:183A58004200B70042A0B7001400F800D68ABF0032A0B700D48ABF00F3
:183A700014A0B700000DBB002004240060A7B70040A7A9004200F8003B
:183A8800000E20004200B70042A0B7005005200066A7B700A00A200063
:183AA00066A7B70061E7A80000000000000000004200F9000060FE00C1
:183AB8001400F900DF6AEF004200F90000C2B300EF4AB50018003A00C1
:183AD00000C0B300DF4AB50015003A004200F800000E20004200B700DD
:183AE80042A0B7001400F800D68ABF0032A0B700D48ABF0014A0B700F1
:183B000000DB20001AA0B7003D007800000DBB003D007800009DBB00B7
:183B18003D007800000DBB003D007800009DBB001400F9004200F900C3
:183B300066003700E09C2000E40ABD000F003A000E00F8000A96BF00EB
:183B480009003200004021000816B4000EA0B70007409000CEE9B7004D
:183B60000A36ED000836EC000936A90002003700CE29EF00CEC9A800B0
:183B78000E00F90000C0B300ED4AB50007003A000400FC003B4078009B
:183B9000BDEAB700BDCABF003A010700F9CABF00D100070010C0B3005A
:183BA800ED4AB5000B003A000400FC003B407800BDEAB7003B40780090
:183BC000BEEAB700BDCABF002E010700BECABF002C010700F8CABF0016
:183BD800C300070020C0B300ED4AB50013003A000800FC003B40780048
:183BF000BDEAB7003B407800BEEAB7003B407800BFEAB7003B407800C7
:183C0800C0EAB700BDCABF001C010700BECABF001A010700BFCABF0028
:183C200018010700C0CABF0016010700F5CABF00AD00070030C0B30030
:183C3800ED4AB50023003A001000FC003B407800BDEAB7003B407800DB
:183C5000BEEAB7003B407800BFEAB7003B407800C0EAB7003B40780063
:183C6800C1EAB7003B407800C2EAB7003B407800C3EAB7003B40780042
:183C8000C4EAB700BDCABF00FE000700BECABF00FC000700BFCABF00EA
:183C9800FA000700C0CABF00F8000700C1CABF00F6000700C2CABF0039
:183CB000F4000700C3CABF00F2000700C4CABF00F0000700F4CABF00FB
:183CC800870007000A409000FA4AB70013FD3A0062CDBF000200320015
:183CE0008BCABF00E70007004889BF004CA9B700C9EAEF00C4C9BF00A0
:183CF8001100320002100700C469EF000E00F8000A96BF00090032009C
:183D1000004021000816B4000EA0B70007409000CEE9B7000A36ED0091
:183D28000836EC000936A90002003700CE29EF00CEC9A8000E00F9000C
:183D4000F4FB37007EA9B7007C09F9007609F9007609F8007C09F8007D
:183D580076A9ED007A29EC000010200078A9B700004006007EA9B7008C
:183D70007C09F9007609F9007609F8007C09F80076A9ED007A29EC00B6
:183D88001000200078A9B700004006007EA9B7007C09F9007609F90001
:183DA0007609F8007C09F80076A9ED007A29EC002000200078A9B70064
:183DB8008060A90040A7A800004006007EA9B7007C09F9007609F900C1
:183DD0007609F8007C09F80076A9ED007A29EC003000200078A9B70024
:183DE80000DC20001EA0B7008040A900004006007EA9B7007C09F90047
:183E00007609F9007609F8007C09F80076A9ED007A29EC004000200043
:183E180078A9B7008080A900004006007EA9B7007C09F9007609F900F7
:183E30007609F8007C09F80076A9ED007A29EC005000200078A9B700A3
:183E4800E083BF007CA9B70080A0A900004006007EA9B7007C09F900F9
:183E60007609F9007609F8007C09F80076A9ED007A29EC0060002000C3
:183E78007CA9B700004006007EA9B7007C09F9007609F9007609F800C5
:183E90007C09F80076A9ED007A29EC00700020007CA9B7000040060050
:183EA800D0C0B30001000700A0C0B3009EEAB7002222A9000060FE001A
:183EC0002322AF00FDFF37009ECABF0024E2B700000006001041230065
:183ED80090A9B7009029ED00FEFF3A0000000600CDEAB700CECABF003A
:183EF0004220AE000700370016C0BF00CD4AB50016E0B70017C0BF00C8
:183F0800FACAB50017E0B7000B00370000C0B3006A4DB50005003A001A
:183F200016C0BF00E4EAB70017C0BF00E5EAB700030037000020EF000A
:183F3800CDCABF00E02AB40000000600C6CABF000A003A004289BF003A
:183F5000040032000028EF000228EF004229EF00542AEF00528ABF0091
:183F680001003200522AEF00F4FF370000D72000B20AB40018A0B700A3
:183F8000003020001C00600009003200CBCABF000700320000C4B3001E
:183F9800614DB70061EDB7000500FC0000DC20001EA0B7005FFB3700A4
:183FB0000C409000ECEAB7001820EC000C409000B8EAB700C66AED001A
:183FC800B2AAEC00B2CAA900ECCABF0000000600C6CABF000A003A0066
:183FE0004289BF00040032000028EF000228EF004229EF00542AEF0012
:183FF800528ABF0001003200522AEF00F4FF370000D72000B20AB400E7
:1840100018A0B700003020001C00600009003200CBCABF000700320095
:1840280000C4B300614DB70061EDB7000500FC0000DC20001EA0B7002D
:184040003AFB37000C409000ECEAB7001820EC000C409000B8EAB7003A
:18405800C66AED00B2AAEC00B2CAA900ECCABF00ECCABF008CEAB600B0
:1840700000F020008C4AB4001040BA008CEAB70000000600ECEAB700D4
:18408800ECCABF0089FF0700ECCABF008BEAB60000F020008B4AB400E3
:1840A0001040BA008BEAB70000000600CAFF0700ECCABF00005D7800B2
:1840B8000000060060C0B300E64AB500060031000020EF00E6CABF007D
:1840D0000020B4000020B40016A0B700010037000B00200030C0B300BD
:1840E800664DB500060031000020EF0066CDBF000020B4000020B40078
:184100000CA0B7000100370006002000C0072B001620B4000B0090006F
:184118008EA9B70016A0EC000B0090000C20B4000600900026AAB70067
:184130000CA0EC00060090008AA9B70060AA2A0028AAB700000006009C
:18414800000020008B49B4008CA9B7008CC9BF0003003200D3FF0700A9
:184160008C29ED00FBFF370062CDBF000C0032008CCABF0073FF0700BA
:18417800ECCABF008C4AB5000700320010C0B300616DB700636DEC0032
:184190000500FC0000DC20001EA0B700E3FA37008B6AEF0000E02000AD
:1841A80014A0B700000006008CA9B7008CC9BF00040032003B40780065
:1841C000B0FF07008C29ED00FAFF3700000006008CA9B7008CC9BF0059
:1841D800040032003A407800805D78008C29ED00FAFF3700000006007A
:1841F000B0000000000000004E6F00004B650000796200006F610000EF
:18420800726400004E6F000044690000737000006C6100007900000035
:18422000B000000001000000496E000070750000744F0000757400008D
:1842380070750000744500006E6300006F640000657200000000000055
:18425000B001000001000000496E000070750000744F0000757400005C
:1842680070750000744500006E6300006F64000065720000416E000076
:18428000616C00006F67000000000000B002000001000000496E000019
:1842980070750000744F00007574000070750000744500006E6300000E
:1842B0006F64000065720000416E0000616C00006F67000000000000FA
:1842C800B0010000000000004E6F00004B650000796200006F61000015
:1842E0007264000044690000737000006C61000079000000B00000006A
:1842F80001000000496E000070750000744F0000757400007075000080
:18431000744500006E6300006F640000657200004469000073700000D1
:184328006C61000079000000B001000001000000496E000070750000E9
:18434000744F00007574000070750000744500006E6300006F64000077
:1843580065720000416E0000616C00006F670000446900007370000094
:184370006C61000079000000B002000001000000496E000070750000A0
:18438800744F00007574000070750000744500006E6300006F6400002F
:1843A00065720000416E0000616C00006F670000576900006465000053
:1843B80044690000737000006C61000079000000B00200000000000065
:1843D0004B650000796200006F6100007264000034620000793800005D
:1843E8004E6F000044690000737000006C61000079000000B00000007A
:1844000001000000496E000070750000744F0000757400007075000076
:18441800744500006E6300006F640000657200004B65000079630000CC
:184430006F640000653400006279000038000000B00100000100000043
:18444800496E000070750000744F000075740000707500007445000076
:184460006E6300006F64000065720000416E0000616C00006F67000077
:184478004B650000796300006F64000065340000627900003800000021
:18449000B002000001000000496E000070750000744F00007574000019
:1844A80070750000744500006E6300006F64000065720000416E000034
:1844C000616C00006F6700004B650000796300006F6400006534000049
:1844D8006279000038000000B0030000000000004B650000796200007B
:1844F0006F610000726400003462000079380000446900007370000037
:184508006C61000079000000B000000001000000496E00007075000008
:18452000744F00007574000070750000744500006E6300006F64000095
:184538006572000044690000737000006C610000794B00006579000095
:18455000636F000064650000346200007938000000000000B0010000C0
:1845680001000000496E000070750000744F000075740000707500000D
:18458000744500006E6300006F64000065720000416E0000616C000073
:184598006F67000044690000737000006C610000794B00006579000036
:1845B000436F000064650000346200007938000000000000B00200007F
:1845C80001000000496E000070750000744F00007574000070750000AD
:1845E000744500006E6300006F64000065720000416E0000616C000013
:1845F8006F670000576900006465000044690000737000006C610000EF
:18461000794B000065790000436F00006465000034620000793800002E
:1846280000000000B0040000000000004B650000796200006F6100006B
:184640007264000038620000793800004E6F00004469000073700000F4
:184658006C61000079000000B000000001000000496E000070750000B7
:18467000744F00007574000070750000744500006E6300006F64000044
:18468800657200004B650000796300006F64000065380000627900006C
:1846A00038000000B001000001000000496E000070750000744F0000B9
:1846B8007574000070750000744500006E6300006F64000065720000E8
:1846D000416E0000616C00006F6700004B650000794300006F64000041
:1846E800653800006279000038000000B002000001000000496E0000A0
:1847000070750000744F00007574000070750000744500006E630000A1
:184718006F64000065720000416E0000616C00006F6700004B650000DD
:18473000794300006F640000653800006279000038000000B00500007D
:18474800000000004B650000796200006F61000072640000386200008E
:184760007938000044690000737000006C61000079000000B00000000A
:1847780001000000496E000070750000744F00007574000070750000FB
:18479000744500006E6300006F6400006572000044690000737000004D
:1847A8006C610000794B000065790000636F0000646500003862000055
:1847C0007938000000000000B001000001000000496E000070750000E2
:1847D800744F00007574000070750000744500006E6300006F640000DB
:1847F00065720000416E0000616C00006F6700004469000073700000F8
:184808006C610000794B000065790000436F0000646500003862000014
:184820007938000000000000B002000001000000496E00007075000080
:18483800744F00007574000070750000744500006E6300006F6400007A
:1848500065720000416E0000616C00006F67000057690000646500009E
:1848680044690000737000006C610000794B000065790000436F000087
:1848800064650000386200007938000000000000A020000006800000C6
:1848980000000000000000000000000000000000940800004E6F0000AF
:1848B0006E6500000044000069730000706C00006179000033320000E2
:1848C80000000000A008000006800000000000000000000000000000AA
:1848E00000000000940800004E6F00006E650000004400006973000074
:1848F800706C00006179000000000000A0080000060000000000000044
:18491000000000000000000000000000CE0900004E6F00006E65000028
:18492800004B000065790000636F00006465000000000000A0160000FD
:18494000018000000000000000000000000000000000000000080000D6
:184958004E6F00006E650000004F000075740000707500007400000026
:18497000A00E0000018000000000000000000000000000000000000000
:18498800000800004E6F00006E650000004F0000757400007075000062
:1849A00074000000A01200000180000000000000000000000000000058
:1849B80000000000000800004E6F00006E650000004F00007574000017
:1849D0007075000074000000A00A00000180000000000000000000004B
:1849E8000000000000000000000800004E6F00006E650000004F0000D0
:184A0000757400007075000074000000A0060000018000000000000035
:184A1800000000000000000000000000000800004E6F00006E650000EE
:184A3000004F0000757400007075000074000000A01800000100000024
:184A480000000000000000000000000000000000080800004E6F000089
:184A60006E650000004900006E7000007574000000000000A0100000AB
:184A780001000000000000000000000000000000000000000808000015
:184A90004E6F00006E650000004900006E70000075740000000000006E
:184AA800A010000008000000000000000000000000000000000000003E
:184AC000A0090000436F0000756E000074730000004500006E630000A3
:184AD80030000000A010000008000000000000000000000000000000DE
:184AF00000000000A2090000436F0000756E0000747300000045000042
:184B08006E63000031000000A0100000080000000000000000000000DB
:184B20000000000000000000A4090000436F0000756E00007473000054
:184B3800004500006E63000032000000A0100000080000000000000065
:184B5000000000000000000000000000A6090000436F0000756E000009
:184B680074730000004500006E63000033000000A00800000800000055
:184B800000000000000000000000000000000000A0090000436F0000C2
:184B9800756E000074730000004500006E63000030000000A00800004D
:184BB0000800000000000000000000000000000000000000A20900003A
:184BC800436F0000756E000074730000004500006E6300003100000012
:184BE000A008000008000000000000000000000000000000000000000D
:184BF800A4090000436F0000756E000074730000004500006E63000066
:184C100032000000A008000008000000000000000000000000000000AA
:184C280000000000A6090000436F0000756E0000747300000045000004
:184C40006E63000033000000A0080000020000000000000000000000AE
:184C5800333300005340000010080000566F00006C740000730000001B
:184C7000416E0000616C00006F670000496E000030000000A00800004B
:184C880002000000000000000000000033330000534000001108000000
:184CA000566F00006C74000073000000416E0000616C00006F67000092
:184CB800496E000031000000A008000002000000000000000000000052
:184CD000333300005340000012080000566F00006C74000073000000A1
:184CE800416E0000616C00006F670000496E000032000000A0080000D1
:184D000002000000000000000000000033330000534000001308000085
:184D1800566F00006C74000073000000416E0000616C00006F67000019
:184D3000496E000033000000A01000000280000000000000000000004F
:184D48000000000000000000C60900004E6F00006E65000000430000B1
:184D60006F6E0000747200006173000074000000A010000002800000FE
:184D780000000000000000000000000000000000980900004E6F0000C5
:184D90006E650000004500006E6300004D6F000064650000300000006D
:184DA800A01000000280000000000000000000000000000000000000C1
:184DC0009A0900004E6F00006E650000004500006E6300004D6F0000D6
:184DD8006465000031000000A010000002800000000000000000000097
:184DF00000000000000000009C0900004E6F00006E6500000045000031
:184E08006E6300004D6F00006465000032000000A010000002800000D8
:184E2000000000000000000000000000000000009E0900004E6F000016
:184E38006E650000004500006E6300004D6F00006465000033000000C1
:184E5000A0100000028000000000000000000000000000000000000018
:184E68005C0900004E6F00006E65000000530000775200006576000046
:184E800069730000696F00006E000000A01000000280000000000000C6
:184E9800000000000000000000000000740900004E6F00006E650000F5
:184EB00000480000775200006576000069730000696F00006E000000DC
:184EC800A01000000280000000000000000000000000000000000000A0
:184EE000DE0900004E6F00006E650000004B0000657900004D6F00005E
:184EF8006465000000000000A0100000048000000000000000000000A5
:184F10000000000000000000440000004E6F00006E650000004E000067
:184F2800564300006F6E0000747200006173000074000000A01000001D
:184F400004800000000000000000000000000000000000003A0000009B
:184F58004E6F00006E650000004E0000564500006E6300004D6F00003B
:184F70006465000030000000A0100000048000000000000000000000FC
:184F880000000000000000003C0000004E6F00006E650000004E0000F7
:184FA000564500006E6300004D6F00006465000031000000A010000027
:184FB80004800000000000000000000000000000000000003E0000001F
:184FD0004E6F00006E650000004E0000564500006E6300004D6F0000C3
:184FE8006465000032000000A010000004800000000000000000000082
:185000000000000000000000400000004E6F00006E650000004E00007A
:18501800564500006E6300004D6F00006465000033000000A0100000AC
:18503000048000000000000000000000000000000000000006000000DE
:185048004E6F00006E650000004E00005644000069730000704D00003F
:185060006F64000065000000A0100000048000000000000000000000CC
:185078000000000000000000460000004E6F00006E650000004E0000FC
:18509000564B000065790000546900006D65000072000000A0100000D8
:1850A8000480000000000000000000000000000000000000420000002A
:1850C0004E6F00006E650000004E0000564100006E6100006C6F0000B9
:1850D80067460000696C00007465000072000000A010000004400000FF
:1850F00000000000000000000000000000000000000000004E6F0000EB
:185108006E650000004E00005642000061750000645200006174000075
:1851200065000000A0200000040000000000000000000000000000004E
:1851380000000000780000004E6F00006E650000004E0000565500005E
:185150006E690000744E0000756D00006265000072000000A0100000E3
:18516800040000000000000000000000000000000000000038000000F3
:185180004E6F00006E650000004E0000565700006174000063680000EC
:18519800446F000067540000696D0000656F00007574000000000000FE
:1851B000F8A0000010A100009EA4000020A5000054A500006EA500008B
:1851C80088A50000A2A5000000000000F8A0000028A100009EA40000B8
:1851E00020A50000BCA50000D6A50000F0A500000AA6000024A6000007
:1851F80042A6000060A600007EA6000000000000F8A0000046A100000E
:185210009EA4000020A50000BCA50000D6A50000F0A500000AA600005E
:1852280024A6000042A6000060A600007EA600000000000064A100008D
:185240007AA1000066A40000B8A4000020A5000054A500006EA5000004
:1852580088A50000A2A500000000000064A1000098A1000066A4000082
:18527000B8A4000020A50000BCA50000D6A50000F0A500000AA60000E4
:1852880024A6000042A6000060A600007EA600000000000064A100002D
:1852A000BCA1000048A40000B8A4000020A50000BCA50000D6A50000B0
:1852B800F0A500000AA6000024A6000042A6000060A600007EA60000BD
:1852D00000000000E4A10000FEA1000082A40000D2A400003AA5000027
:1852E80054A500006EA5000088A50000A2A5000000000000E4A10000A9
:1853000020A2000082A40000D2A400003AA50000BCA50000D6A500007C
:18531800F0A500000AA6000024A6000042A6000060A600007EA600005C
:1853300000000000E4A1000048A2000082A40000D2A400003AA500007B
:18534800BCA50000D6A50000F0A500000AA6000024A6000042A600007A
:1853600060A600007EA600000000000070A2000088A2000066A40000C5
:1853780082A40000ECA400003AA5000054A500006EA5000088A500004F
:18539000A2A500000000000070A20000B2A2000066A4000082A4000028
:1853A800ECA400003AA50000BCA50000D6A50000F0A500000AA600005D
:1853C00024A6000042A6000060A600007EA600000000000070A20000E7
:1853D800E2A2000048A4000082A40000ECA400003AA50000BCA5000057
:1853F000D6A50000F0A500000AA6000024A6000042A6000060A600002D
:185408007EA600000000000016A3000030A3000082A40000B8A400005A
:185420003AA5000054A500006EA5000088A50000A2A500000000000015
:1854380016A3000052A3000082A40000B8A400003AA50000BCA50000EC
:18545000D6A50000F0A500000AA6000024A6000042A6000060A60000CC
:185468007EA600000000000016A300007AA3000082A40000B8A40000B0
:185480003AA50000BCA50000D6A50000F0A500000AA6000024A600004A
:1854980042A6000060A600007EA6000000000000A2A30000BAA3000048
:1854B00066A4000082A4000006A500003AA5000054A500006EA500001E
:1854C80088A50000A2A5000000000000A2A30000E4A3000066A4000082
:1854E00082A4000006A500003AA50000BCA50000D6A50000F0A5000093
:1854F8000AA6000024A6000042A6000060A600007EA600000000000010
:18551000A2A3000014A4000048A4000082A4000006A500003AA50000EA
:18552800BCA50000D6A50000F0A500000AA6000024A6000042A6000098
:1855400060A600007EA6000000000000F8A0000010A1000028A1000017
:1855580046A1000064A100007AA1000098A10000BCA10000E4A1000019
:18557000FEA1000020A2000048A2000070A2000088A20000B2A2000048
:18558800E2A2000016A3000030A3000052A300007AA30000A2A30000A4
:1855A000BAA30000E4A3000014A4000048A4000066A4000082A400003B
:1855B8009EA40000B8A40000D2A40000ECA4000006A5000020A50000C7
:1855D0003AA5000054A500006EA5000088A50000A2A50000BCA5000003
:1855E800D6A50000F0A500000AA6000024A6000042A6000060A6000033
:185600007EA600009CA60000B8A60000D4A60000F0A600000CA700000B
:1856180028A7000046A7000064A7000080A700009EA70000BCA70000E4
:18563000DAA70000F8A7000016A8000034A8000052A8000074A8000092
:1856480092A80000B2A8000000000000BCFA07000B942000100020000A
:18566000D3FA07000B80200030002000D8FA07008B802000300020000F
:18567800CDFA07000B9A200020002000CAFA07002B9A20002000200057
:18569000C7FA07004B9A200020002000C4FA07006B9A200020002000CB
:1856A800C1FA07008AF93700A5FA07000B94200010002000BCFA07001C
:1856C0000B80200030002000C1FA07008B80200030002000B6FA0700E3
:1856D8000B9A200010002000B3FA07002B9A200010002000B0FA07004B
:1856F0004B9A200010002000ADFA07006B9A200010002000AAFA0700BF
:185708000B81200010002000A7FA07001B81200010002000A4FA070074
:185720002B81200010002000A1FA07003B812000100020009EFA070028
:1857380067F9370082FA07000B9420001000200099FA07000B8020000B
:18575000300020009EFA07008B8020003000200093FA07000B9A20007E
:185768001000200090FA07002B9A2000100020008DFA07004B9A2000C0
:18578000100020008AFA07006B9A20001000200087FA07000B812000CD
:185798001000200084FA07001B8120001000200081FA07002B8120000A
:1857B000100020007EFA07003B812000100020007BFA070044F9370036
:1857C8005FFA07000B9420001000200076FA07004B89200010002000DF
:1857E0007BFA07000B8020002000200078FA07008B8020003000200056
:1857F8006DFA07000B9A2000200020006AFA07002B9A20002000200096
:1858100067FA07004B9A20002000200064FA07006B9A20002000200009
:1858280061FA07002AF9370045FA07000B942000100020005CFA07001A
:185840004B8920001000200061FA07000B802000200020005EFA070080
:185858008B8020003000200053FA07000B9A20001000200050FA070023
:185870002B9A2000100020004DFA07004B9A2000100020004AFA07003D
:185888006B9A20001000200047FA07000B8120001000200044FA07004A
:1858A0001B8120001000200041FA07002B812000100020003EFA070087
:1858B8003B812000100020003BFA070004F937001FFA07000B9420007D
:1858D0001000200036FA07004B892000400020003BFA07000B8020001E
:1858E8002000200038FA07008B802000300020002DFA07000B9A2000C1
:18590000100020002AFA07002B9A20001000200027FA07004B9A2000F2
:185918001000200024FA07006B9A20001000200021FA07000B812000FF
:18593000100020001EFA07001B812000100020001BFA07002B8120003C
:185948001000200018FA07003B8120001000200015FA0700DEF83700CF
:18596000F9F907000B9420001000200010FA0700EB9C2000100020005F
:185978000DFA07000B8020003000200012FA07008B8020002000200090
:1859900007FA07000B9A20002000200004FA07002B9A200020002000C8
:1859A80001FA07004B9A200020002000FEF907006B9A2000200020003D
:1859C000FBF90700C4F83700DFF907000B94200010002000F6F907001D
:1859D800EB9C200010002000F3F907000B80200030002000F8F90700FA
:1859F0008B80200020002000EDF907000B9A200010002000EAF9070068
:185A08002B9A200010002000E7F907004B9A200010002000E4F9070071
:185A20006B9A200010002000E1F907000B81200010002000DEF907007E
:185A38001B81200010002000DBF907002B81200010002000D8F90700BB
:185A50003B81200010002000D5F907009EF83700B9F907000B94200018
:185A680010002000D0F90700EB9C200010002000CDF907000B802000D7
:185A800030002000D2F907008B80200020002000C7F907000B9A2000F5
:185A980010002000C4F907002B9A200010002000C1F907004B9A200027
:185AB00010002000BEF907006B9A200010002000BBF907000B81200034
:185AC80010002000B8F907001B81200010002000B5F907002B81200071
:185AE00010002000B2F907003B81200010002000AFF9070078F837006A
:185AF80093F907000B94200010002000AAF907004B8920001000200046
:185B1000AFF90700EB9C200010002000A4F907000B8020002000200068
:185B2800A9F907008B802000200020009EF907000B9A200020002000AE
:185B40009BF907002B9A20002000200098F907004B9A200020002000B0
:185B580095F907006B9A20002000200092F907005BF8370076F90700A9
:185B70000B942000100020008DF907004B8920001000200092F90700EB
:185B8800EB9C20001000200087F907000B802000200020008CF9070030
:185BA0008B8020002000200081F907000B9A2000100020007EF907008E
:185BB8002B9A2000100020007BF907004B9A20001000200078F9070098
:185BD0006B9A20001000200075F907000B8120001000200072F90700A5
:185BE8001B812000100020006FF907002B812000100020006CF90700E2
:185C00003B8120001000200069F9070032F837004DF907000B942000AA
:185C18001000200064F907004B8920004000200069F90700EB9C20007C
:185C3000100020005EF907000B8020002000200063F907008B80200055
:185C48002000200058F907000B9A20001000200055F907002B9A20007D
:185C60001000200052F907004B9A2000100020004FF907006B9A200001
:185C7800100020004CF907000B8120001000200049F907001B812000B7
:185C90001000200046F907002B8120001000200043F907003B8120006B
:185CA8001000200040F9070009F8370024F907000B9420001000200029
:185CC0003BF90700EB9C20001000200038F907000B8020002000200097
:185CD8003DF907008B8020002000200032F907000B9A200020002000D5
:185CF0002FF907002B9A2000200020002CF907004B9A200020002000D7
:185D080029F907006B9A20002000200026F90700EFF737000AF90700A8
:185D20000B9420001000200021F90700EB9C2000100020001EF9070066
:185D38000B8020002000200023F907008B8020002000200018F90700C2
:185D50000B9A20001000200015F907002B9A20001000200012F907000A
:185D68004B9A2000100020000FF907006B9A2000100020000CF907007E
:185D80000B8120001000200009F907001B8120001000200006F9070034
:185D98002B8120001000200003F907003B8120001000200000F90700E8
:185DB000C9F73700E4F807000B94200010002000FBF80700EB9C200071
:185DC80010002000F8F807000B80200020002000FDF807008B8020008A
:185DE00020002000F2F807000B9A200010002000EFF807002B9A2000B2
:185DF80010002000ECF807004B9A200010002000E9F807006B9A200036
:185E100010002000E6F807000B81200010002000E3F807001B812000EB
:185E280010002000E0F807002B81200010002000DDF807003B8120009F
:185E400010002000DAF80700A3F73700BEF807000B94200010002000C4
:185E5800D5F807004B89200010002000DAF80700EB9C2000100020008A
:185E7000CFF807000B80200010002000D4F807008B8020002000200033
:185E8800C9F807000B9A200020002000C6F807002B9A2000200020004B
:185EA000C3F807004B9A200020002000C0F807006B9A200020002000BF
:185EB800BDF8070086F73700A1F807000B94200010002000B8F807001C
:185ED0004B89200010002000BDF80700EB9C200010002000B2F8070052
:185EE8000B80200010002000B7F807008B80200020002000ACF80700FB
:185F00000B9A200010002000A9F807002B9A200010002000A6F8070032
:185F18004B9A200010002000A3F807006B9A200010002000A0F80700A6
:185F30000B812000100020009DF807001B812000100020009AF807005C
:185F48002B8120001000200097F807003B8120001000200094F8070010
:185F60005DF7370078F807000B942000100020008FF807004B892000B6
:185F78004000200094F80700EB9C20001000200089F807000B80200014
:185F9000100020008EF807008B8020002000200083F807000B9A20008A
:185FA8001000200080F807002B9A2000100020007DF807004B9A20009C
:185FC000100020007AF807006B9A20001000200077F807000B812000A9
:185FD8001000200074F807001B8120001000200071F807002B812000E6
:185FF000100020006EF807003B812000100020006BF8070034F7370024
:18600800D8A800000C030000EAA800000C03000004A900000C03000094
:18602000000000001EA900000C03000032A900000C0300004EA90000B1
:186038000C060000000000006AA900000C0300007EA900000C030000E6
:186050009AA900000C03000000000000B6A900000C030000CCA9000003
:186068000C030000EAA900000C0600000000000008AA00000C020000AC
:186080001CAA00000C02000038AA00000C0200000000000054AA000046
:186098000C0200006AAA00000C02000088AA00000C050000000000007D
:1860B0002A2B0000582B00009E2B0000E42B0000182C0000642C000054
:1860C800B02C0000E42C0000302D00007C2D0000B62D0000082E0000B5
:1860E0005A2E00008E2E0000DA2E0000262F0000602F0000B22F000097
:1860F80058B0000004B000005EB0000012B0000064B0000020B0000020
:186110006AB000002EB0000070B000003CB0000076B000004AB0000053
:18612800000000008560A9000000F8001000F80026C2BF008AEAB700FF
:1861400000042000C64AB5001100320000D72000B40AB40010A0B7004B
:186158008ACABF00004498001020EC0084E0AE000200370010C0B30056
:186170000100370000C0B300004498000621EF0084E0A900C66AEC0051
:18618800B4AAEC00B4CAA9002202AF00E8FF37001000F9000000F9009B
:1861A000004006000000F8000000F9008C20A900004006000000F8001D
:1861B80094E0A900B7EAEF0011E1A9000000F90084E0A900004006003B
:1861D0000000F8000000F9008760A900004006000060FE000000F8009A
:1861E80000002000C209BD00500032007E8ABF004D003A000E00F80021
:1862000020C0B3007B4AB50012003A00BF09AE0002003700ECC2A80028
:1862180001003700ECC2A900BEC9BF00B8E9B700000F2000CD42B6004D
:18623000B9E9B700F0002000B849B600B949B700CDE2B700F442A80039
:18624800100020007BEAB7003500370030C0B3007B4AB50004003A002B
:18626000F442A900200020007BEAB7002E00370000C0B3007B4AB50099
:186278001D003A000496BF001A003200000021000216B4000EA0B700C0
:1862900007009000BEA9B700BF09AE0002003700ECC2A8000100370004
:1862A800ECC2A900BEC9BF0000C0FD00B8E9B700000F2000CD42B60038
:1862C000B9E9B700F0002000B849B600B949B700CDE2B7003000200037
:1862D8007BEAB70004B6ED0002B6EC000356A900F442A8000E00370022
:1862F00010C0B3007B4AB5000B003A00F442A900000020007BEAB70039
:18630800BFE9AE0003003700F07C20007EAAB7000200370050002000D9
:186320007EAAB700000037000E00F900010037007E2AED002A8ABF0008
:18633800080032002A2AED0002003A00F01F20002CAAB7002D2AAF00D4
:18635000EC02A9002D2AAE00EC02A800B089BF00B429B400B289BF0080
:18636800B6A9B4004889BF004A09BD00020032004889BF004CA9B700FA
:186380004C89BF00040032004C29ED0002003A00100020004029B7004D
:186398004889BF004AA9B70000C0B300E249B50038003A000908A90034
:1863B000DA02AF000908A8000928A900DA22AF000928A8000948A90039
:1863C800DA42AF000948A8000968A900DA62AF000968A800DA82BF00C0
:1863E00094A9B7009229A9009409AF009229A8009249A9009609AF00CC
:1863F8009249A8009269A9009429AF009269A8009289A9009629AF0025
:186410009289A80040652C009209B4000EA0B7009889BF004500DD002A
:186428000E20B40007009000A029B4009229A9009449AF009229A80013
:186440009249A9009649AF009249A8009269A9009469AF009269A800BC
:186458009289A9009669AF009289A80040652C009209B4000EA0B70072
:186470009A89BF004500DD000E20B40007009000A229B400E229EC0021
:186488003B00370010C0B300E249B50038003A000988A900DB02AF00EF
:1864A0000988A80009A8A900DB22AF0009A8A80009C8A900DB42AF0006
:1864B80009C8A80009E8A900DB62AF0009E8A8009229A9009509AF0083
:1864D0009229A8009249A9009709AF009249A8009269A9009529AF00EA
:1864E8009269A8009289A9009729AF009289A80040652C009209B400E3
:186500000EA0B7009C89BF004500DD000E20B40007009000A429B4001E
:186518009229A9009549AF009229A8009249A9009749AF009249A80081
:186530009269A9009569AF009269A8009289A9009769AF009289A80029
:1865480040652C009209B4000EA0B7009E89BF004500DD000E20B400CC
:1865600007009000A629B4009489BF0096A9B700E229EF000000370006
:1865780000C0B300C849B50086003A000AA3A8000BA3A8000CA3A80010
:186590000DA3A80000C0B300E049B5000D003A0041C3BF0010E8B70091
:1865A80000C9B3001048B500020039000808A8000400370090C6B3001B
:1865C0001048B500010031000808A900E029EC007000370010C0B300AC
:1865D800E049B5000D003A0043C3BF0011E8B70000C9B3001148B50087
:1865F000020039000828A8000400370090C6B3001148B50001003100FC
:186608000828A900E029EC006000370020C0B300E049B5000D003A005D
:1866200045C3BF0012E8B70000C9B3001248B500020039000848A8002C
:186638000400370090C6B3001248B500010031000848A900E029EC00D7
:186650005000370030C0B300E049B5000D003A0047C3BF0013E8B70068
:1866680000C9B3001348B500020039000868A8000400370090C6B300F7
:186680001348B500010031000868A900E029EC004000370040C0B30088
:18669800E049B5000D003A0049C3BF0014E8B70000C9B3001448B500BA
:1866B000020039000888A8000400370090C6B3001448B50001003100D8
:1866C8000888A900E029EC003000370050C0B300E049B5000D003A003D
:1866E0004BC3BF0015E8B70000C9B3001548B5000200390008A8A80000
:1866F8000400370090C6B3001548B5000100310008A8A900E029EC00B4
:186710002000370060C0B300E049B5000D003A004DC3BF0016E8B7009E
:1867280000C9B3001648B5000200390008C8A8000400370090C6B300D3
:186740001648B5000100310008C8A900E029EC001000370070C0B30064
:18675800E049B5000D003A004FC3BF0017E8B70000C9B3001748B500ED
:186770000200390008E8A8000400370090C6B3001748B50001003100B4
:1867880008E8A900E029EF0000003700C829EC005805370010C0B3003D
:1867A000C849B50031053A0010C0B300DE49B50053023A0000C0B3004A
:1867B800D449B5001C003A00F102A900D609A800CBC2AF00D609A900BA
:1867D000D629A800CBE2AF00D629A900D649A800EA82AF00D649A9005C
:1867E800D669A800EAA2AF00D669A900D689A800DAA2AF00D689A90055
:18680000D6A9A800DAE2AF00D6A9A900D6C9A800E222AF00D6C9A90084
:18681800D6E9A800E262AF00D6E9A900F102A800D429EC0033023700B6
:1868300010C0B300D449B5001C003A00F122A900D709A800CBC2AF0025
:18684800D709A900D729A800CBE2AF00D729A900D749A800EA82AF001F
:18686000D749A900D769A800EAA2AF00D769A900D789A800DAA2AF0018
:18687800D789A900D7A9A800DAE2AF00D7A9A900D7C9A800E222AF0048
:18689000D7C9A900D7E9A800E262AF00D7E9A900F122A800D429EC003F
:1868A8001402370020C0B300D449B5001C003A00C982A900D809A80053
:1868C000CBC2AF00D809A900D829A800CBE2AF00D829A900D849A80082
:1868D800EA82AF00D849A900D869A800EAA2AF00D869A900D889A800AC
:1868F000DAA2AF00D889A900D8A9A800DAE2AF00D8A9A900D8C9A80054
:18690800E222AF00D8C9A900D8E9A800E262AF00D8E9A900C982A800C1
:18692000D429EC00F501370030C0B300D449B5001C003A00C9A2A9006A
:18693800D909A800CBC2AF00D909A900D929A800CBE2AF00D929A90045
:18695000D949A800EA82AF00D949A900D969A800EAA2AF00D969A9006F
:18696800D989A800DAA2AF00D989A900D9A9A800DAE2AF00D9A9A90017
:18698000D9C9A800E222AF00D9C9A900D9E9A800E262AF00D9E9A900EF
:18699800C9A2A800D429EC00D601370040C0B300D449B50006003A0018
:1869B000D689BF000CB6B700D889BF000EB6B700D429EC00CD013700AF
:1869C80050C0B300D449B50006003A00DA89BF0010B6B700DC89BF001F
:1869E00012B6B700D429EC00C401370060C0B300D449B500B9003A00A3
:1869F800D689BF001496B60008003A00D889BF001696B60005003A0006
:186A1000DA89BF001896B60002003A00DC89BF001A96B600A2003A0046
:186A28000C96BF0002A0B7000000CF004200AF00060037000020ED0092
:186A40004200A9000100AD000280BF000CB6B700200037000E96BF0031
:186A580002A0B7000000CF004200AF00060037000020ED004200A900D8
:186A70000100AD000280BF000EB6B700150037001096BF0002A0B7009A
:186A88000000CF004200AF00060037000020ED004200A9000100AD0053
:186AA0000280BF0010B6B7000A0037001296BF0002A0B7000000CF0050
:186AB8004200AF00050037000020ED004200A9000100AD000280BF00B2
:186AD00012B6B7004200AF00600037000C96BF0002A0B7000000CF001E
:186AE8004200AF00060037000020ED004200A9000100AD000280BF0081
:186B00000CB6B700200037000E96BF0002A0B7000000CF004200AF0031
:186B1800060037000020ED004200A9000100AD000280BF000EB6B700C6
:186B3000150037001096BF0002A0B7000000CF004200AF000600370046
:186B48000020ED004200A9000100AD000280BF0010B6B7000A00370090
:186B60001296BF0002A0B7000000CF004200AF00050037000020ED0054
:186B78004200A9000100AD000280BF0012B6B7004200AF003100370053
:186B90000C96BF0002A0B7000000CF004200AF00060037000020ED0029
:186BA8004200A9000100AD000280BF000CB6B700200037000E96BF00C8
:186BC00002A0B7000000CF004200AF00060037000020ED004200A9006F
:186BD8000100AD000280BF000EB6B700150037001096BF0002A0B70031
:186BF0000000CF004200AF00060037000020ED004200A9000100AD00EA
:186C08000280BF0010B6B7000A0037001296BF0002A0B7000000CF00E6
:186C20004200AF00050037000020ED004200A9000100AD000280BF0048
:186C380012B6B7004200AF00020037004220A800010037004220A9004E
:186C5000010037004220A900010037004220A90011003200788ABF00A2
:186C6800CA09BD000D003200CA29EC00788ABF00CA09BD0009003A00D2
:186C8000D3E9A800D689BF0070AAB700D889BF0072AAB700DA89BF0094
:186C980074AAB700DC89BF0076AAB70001003700CA29EF0001003700C2
:186CB000CA29EF00D689BF0014B6B700D889BF0016B6B700DA89BF0086
:186CC80018B6B700DC89BF001AB6B700D429EC000801370070C0B30078
:186CE000D449B50002003A00D429EC000301370080C0B300D449B500A5
:186CF80000013A00D3E9AE00FB00370000002000D0A9B700100020002D
:186D10001EB6B7001C36EF00708ABF00688AB6001E16B6002B003200F7
:186D2800708ABF001E16B60015003A00D0C9BF00D2E9B700D2E9A80034
:186D4000D2C9A9000C00F8000B36AF0009003700004021000616B40092
:186D58000CA0B700D2C9BF00004398000A36EC000636EC000736A90051
:186D7000000037000C00F900F0FF2F001E96B600682AB60013003700B5
:186D8800D0C9BF00D2E9B700D2E9A800D2C9A8000C00F8000B36AF008F
:186DA00009003700004021000616B4000CA0B700D2C9BF0000439800D2
:186DB8000A36EC000636EC000736A900000037000C00F9001E96BF00DA
:186DD000682AB700D029EC001C36EC001E96BF001E36B4001C96AE0064
:186DE800CBFF370000012000D0A9B700100020001EB6B7001C36EF0045
:186E0000728ABF006A8AB6001E16B6002B003200728ABF001E16B60029
:186E180015003A00D0C9BF00D2E9B700D2E9A800D2C9A9000C00F8009E
:186E30000B36AF0009003700004021000616B4000CA0B700D2C9BF002C
:186E4800004398000A36EC000636EC000736A900000037000C00F900E1
:186E6000F0FF2F001E96B6006A2AB60013003700D0C9BF00D2E9B70034
:186E7800D2E9A800D2C9A8000C00F8000B36AF000900370000402100C7
:186E90000616B4000CA0B700D2C9BF00004398000A36EC000636EC002E
:186EA8000736A900000037000C00F9001E96BF006A2AB700D029EC000D
:186EC0001C36EC001E96BF001E36B4001C96AE00CBFF3700000220007E
:186ED800D0A9B700100020001EB6B7001C36EF00748ABF006C8AB6000D
:186EF0001E16B6002B003200748ABF001E16B60015003A00D0C9BF00F5
:186F0800D2E9B700D2E9A800D2C9A9000C00F8000B36AF000900370024
:186F2000004021000616B4000CA0B700D2C9BF00004398000A36EC0064
:186F38000636EC000736A900000037000C00F900F0FF2F001E96B6006F
:186F50006C2AB60013003700D0C9BF00D2E9B700D2E9A800D2C9A80023
:186F68000C00F8000B36AF0009003700004021000616B4000CA0B70049
:186F8000D2C9BF00004398000A36EC000636EC000736A9000000370053
:186F98000C00F9001E96BF006C2AB700D029EC001C36EC001E96BF0086
:186FB0001E36B4001C96AE00CBFF370000032000D0A9B70010002000DD
:186FC8001EB6B7001C36EF00768ABF006E8AB6001E16B6002B00320031
:186FE000768ABF001E16B60015003A00D0C9BF00D2E9B700D2E9A80074
:186FF800D2C9A9000C00F8000B36AF0009003700004021000616B400D8
:187010000CA0B700D2C9BF00004398000A36EC000636EC000736A90096
:18702800000037000C00F900F0FF2F001E96B6006E2AB60013003700F4
:18704000D0C9BF00D2E9B700D2E9A800D2C9A8000C00F8000B36AF00D4
:1870580009003700004021000616B4000CA0B700D2C9BF000043980017
:187070000A36EC000636EC000736A900000037000C00F9001E96BF001F
:187088006E2AB700D029EC001C36EC001E96BF001E36B4001C96AE00A3
:1870A000CBFF3700708ABF00720AB700740AB700760AB7000E003A0037
:1870B800D269EF000C00F8000B36AF0009003700004021000616B40031
:1870D0000CA0B700D2C9BF00004398000A36EC000636EC000736A900D6
:1870E800000037000C00F900D3E9A900D429EF0000003700D9023700BA
:1871000020C0B300DE49B500BB023A0000C0B300D449B5001C003A0076
:18711800E0A2A900D609A800CBC2AF00D609A900D629A800CBE2AF00E6
:18713000D629A900D649A800EA82AF00D649A900D669A800EAA2AF00D3
:18714800D669A900D689A800DAA2AF00D689A900D6A9A800DAE2AF007B
:18716000D6A9A900D6C9A800E222AF00D6C9A900D6E9A800E262AF0053
:18717800D6E9A900E0A2A800D429EC009B02370010C0B300D449B5005B
:187190001C003A00E0E2A900D709A800CBC2AF00D709A900D729A80031
:1871A800CBE2AF00D729A900D749A800EA82AF00D749A900D769A80036
:1871C000EAA2AF00D769A900D789A800DAA2AF00D789A900D7A9A8002F
:1871D800DAE2AF00D7A9A900D7C9A800E222AF00D7C9A900D7E9A8005F
:1871F000E262AF00D7E9A900E0E2A800D429EC007C02370020C0B30090
:18720800D449B5001C003A00F0C2A900D809A800CBC2AF00D809A9009C
:18722000D829A800CBE2AF00D829A900D849A800EA82AF00D849A900F9
:18723800D869A800EAA2AF00D869A900D889A800DAA2AF00D889A900F2
:18725000D8A9A800DAE2AF00D8A9A900D8C9A800E222AF00D8C9A90022
:18726800D8E9A800E262AF00D8E9A900F0C2A800D429EC005D0237006F
:1872800030C0B300D449B5001C003A00F0E2A900D909A800CBC2AF00EA
:18729800D909A900D929A800CBE2AF00D929A900D949A800EA82AF00BD
:1872B000D949A900D969A800EAA2AF00D969A900D989A800DAA2AF00B6
:1872C800D989A900D9A9A800DAE2AF00D9A9A900D9C9A800E222AF00E6
:1872E000D9C9A900D9E9A800E262AF00D9E9A900F0E2A800D429EC0020
:1872F8003E02370040C0B300D449B5001C003A00F102A900DA09A80005
:18731000CBC2AF00DA09A900DA29A800CBE2AF00DA29A900DA49A8001F
:18732800EA82AF00DA49A900DA69A800EAA2AF00DA69A900DA89A80049
:18734000DAA2AF00DA89A900DAA9A800DAE2AF00DAA9A900DAC9A800F1
:18735800E222AF00DAC9A900DAE9A800E262AF00DAE9A900F102A800B9
:18737000D429EC001F02370050C0B300D449B5001C003A00F122A9001D
:18738800DB09A800CBC2AF00DB09A900DB29A800CBE2AF00DB29A900E3
:1873A000DB49A800EA82AF00DB49A900DB69A800EAA2AF00DB69A9000D
:1873B800DB89A800DAA2AF00DB89A900DBA9A800DAE2AF00DBA9A900B5
:1873D000DBC9A800E222AF00DBC9A900DBE9A800E262AF00DBE9A9008D
:1873E800F122A800D429EC000002370060C0B300D449B5001C003A00B5
:18740000C982A900DC09A800CBC2AF00DC09A900DC29A800CBE2AF0020
:18741800DC29A900DC49A800EA82AF00DC49A900DC69A800EAA2AF00D0
:18743000DC69A900DC89A800DAA2AF00DC89A900DCA9A800DAE2AF0078
:18744800DCA9A900DCC9A800E222AF00DCC9A900DCE9A800E262AF0050
:18746000DCE9A900C982A800D429EC00E101370070C0B300D449B500FC
:187478001C003A00C9A2A900DD09A800CBC2AF00DD09A900DD29A8008B
:18749000CBE2AF00DD29A900DD49A800EA82AF00DD49A900DD69A80033
:1874A800EAA2AF00DD69A900DD89A800DAA2AF00DD89A900DDA9A8002C
:1874C000DAE2AF00DDA9A900DDC9A800E222AF00DDC9A900DDE9A8005C
:1874D800E262AF00DDE9A900C9A2A800D429EC00C201370080C0B30051
:1874F000D449B500BF013A00D689BF000CB6B700D889BF000EB6B70086
:18750800DA89BF0010B6B700DC89BF0012B6B700D689BF001496B600AB
:1875200008003A00D889BF001696B60005003A00DA89BF001896B600CA
:1875380002003A00DC89BF001A96B600A2003A000C96BF0002A0B700DF
:187550000000CF004200AF00060037000020ED004200A9000100AD0080
:187568000280BF000CB6B700200037000E96BF0002A0B7000000CF006F
:187580004200AF00060037000020ED004200A9000100AD000280BF00DE
:187598000EB6B700150037001096BF0002A0B7000000CF004200AF0096
:1875B000060037000020ED004200A9000100AD000280BF0010B6B70022
:1875C8000A0037001296BF0002A0B7000000CF004200AF0005003700AE
:1875E0000020ED004200A9000100AD000280BF0012B6B7004200AF003C
:1875F800600037000C96BF0002A0B7000000CF004200AF00060037002D
:187610000020ED004200A9000100AD000280BF000CB6B70020003700AB
:187628000E96BF0002A0B7000000CF004200AF00060037000020ED0084
:187640004200A9000100AD000280BF000EB6B700150037001096BF002C
:1876580002A0B7000000CF004200AF00060037000020ED004200A900CC
:187670000100AD000280BF0010B6B7000A0037001296BF0002A0B70095
:187688000000CF004200AF00050037000020ED004200A9000100AD0048
:1876A0000280BF0012B6B7004200AF00310037000C96BF0002A0B700FF
:1876B8000000CF004200AF00060037000020ED004200A9000100AD0017
:1876D0000280BF000CB6B700200037000E96BF0002A0B7000000CF0006
:1876E8004200AF00060037000020ED004200A9000100AD000280BF0075
:187700000EB6B700150037001096BF0002A0B7000000CF004200AF002C
:18771800060037000020ED004200A9000100AD000280BF0010B6B700B8
:187730000A0037001296BF0002A0B7000000CF004200AF000500370044
:187748000020ED004200A9000100AD000280BF0012B6B7004200AF00D2
:18776000020037004220A800010037004220A900010037004220A90048
:18777800010037004220A90011003200788ABF00CA09BD000D003200E3
:18779000CA29EC00788ABF00CA09BD0009003A00D3E9A800D689BF00EC
:1877A80070AAB700D889BF0072AAB700DA89BF0074AAB700DC89BF00EA
:1877C00076AAB70001003700CA29EF0001003700CA29EF00D689BF0088
:1877D80014B6B700D889BF0016B6B700DA89BF0018B6B700DC89BF00AA
:1877F0001AB6B700D3E9AE00FB00370000002000D0A9B70010002000DE
:187808001EB6B7001C36EF00708ABF00688AB6001E16B6002B003200F4
:18782000708ABF001E16B60015003A00D0C9BF00D2E9B700D2E9A80031
:18783800D2C9A9000C00F8000B36AF0009003700004021000616B4008F
:187850000CA0B700D2C9BF00004398000A36EC000636EC000736A9004E
:18786800000037000C00F900F0FF2F001E96B600682AB60013003700B2
:18788000D0C9BF00D2E9B700D2E9A800D2C9A8000C00F8000B36AF008C
:1878980009003700004021000616B4000CA0B700D2C9BF0000439800CF
:1878B0000A36EC000636EC000736A900000037000C00F9001E96BF00D7
:1878C800682AB700D029EC001C36EC001E96BF001E36B4001C96AE0061
:1878E000CBFF370000012000D0A9B700100020001EB6B7001C36EF0042
:1878F800728ABF006A8AB6001E16B6002B003200728ABF001E16B60027
:1879100015003A00D0C9BF00D2E9B700D2E9A800D2C9A9000C00F8009B
:187928000B36AF0009003700004021000616B4000CA0B700D2C9BF0029
:18794000004398000A36EC000636EC000736A900000037000C00F900DE
:18795800F0FF2F001E96B6006A2AB60013003700D0C9BF00D2E9B70031
:18797000D2E9A800D2C9A8000C00F8000B36AF000900370000402100C4
:187988000616B4000CA0B700D2C9BF00004398000A36EC000636EC002B
:1879A0000736A900000037000C00F9001E96BF006A2AB700D029EC000A
:1879B8001C36EC001E96BF001E36B4001C96AE00CBFF3700000220007B
:1879D000D0A9B700100020001EB6B7001C36EF00748ABF006C8AB6000A
:1879E8001E16B6002B003200748ABF001E16B60015003A00D0C9BF00F2
:187A0000D2E9B700D2E9A800D2C9A9000C00F8000B36AF000900370021
:187A1800004021000616B4000CA0B700D2C9BF00004398000A36EC0061
:187A30000636EC000736A900000037000C00F900F0FF2F001E96B6006C
:187A48006C2AB60013003700D0C9BF00D2E9B700D2E9A800D2C9A80020
:187A60000C00F8000B36AF0009003700004021000616B4000CA0B70046
:187A7800D2C9BF00004398000A36EC000636EC000736A9000000370050
:187A90000C00F9001E96BF006C2AB700D029EC001C36EC001E96BF0083
:187AA8001E36B4001C96AE00CBFF370000032000D0A9B70010002000DA
:187AC0001EB6B7001C36EF00768ABF006E8AB6001E16B6002B0032002E
:187AD800768ABF001E16B60015003A00D0C9BF00D2E9B700D2E9A80071
:187AF000D2C9A9000C00F8000B36AF0009003700004021000616B400D5
:187B08000CA0B700D2C9BF00004398000A36EC000636EC000736A90093
:187B2000000037000C00F900F0FF2F001E96B6006E2AB60013003700F1
:187B3800D0C9BF00D2E9B700D2E9A800D2C9A8000C00F8000B36AF00D1
:187B500009003700004021000616B4000CA0B700D2C9BF000043980014
:187B68000A36EC000636EC000736A900000037000C00F9001E96BF001C
:187B80006E2AB700D029EC001C36EC001E96BF001E36B4001C96AE00A0
:187B9800CBFF3700708ABF00720AB700740AB700760AB7000E003A0034
:187BB000D269EF000C00F8000B36AF0009003700004021000616B4002E
:187BC8000CA0B700D2C9BF00004398000A36EC000636EC000736A900D3
:187BE000000037000C00F900D3E9A900D429EF00000037001B00370077
:187BF80000C0B300DE49B50018003A000A08A900CBC2AF000A08A80023
:187C10000A28A900CBE2AF000A28A8000A48A900EA82AF000A48A8003B
:187C28000A68A900EAA2AF000A68A8000A88A900DAA2AF000A88A80034
:187C40000AA8A900DAE2AF000AA8A8000AC8A900E222AF000AC8A80064
:187C58000AE8A900E262AF000AE8A800C829EC002400370020C0B30021
:187C7000C849B50021003A0067CDBF00060032004689BF0004003A00E4
:187C88004029EF00542AEF004229EF0052AAEF0030C0B300664DB500CF
:187CA00002003900000420004029B7004089BF0002003A00EC22A800D3
:187CB800070037000028EF000228EF00EC22A900548ABF0002003A00B6
:187CD00042A9EF0054AAEF00528ABF0003003A004689BF00010032003C
:187CE800676DEF0067CDBF0046E9B700C829EF00000037000000F900D8
:187D00008780A900004006000008AF00D5A2A8000008AE00D5A2A900C9
:187D18000028AF00DCC2A8000028AE00DCC2A9000048AF00E402A80094
:187D30000048AE00E402A9000068AF00E442A8000068AE00E442A900EC
:187D48000088AF00E482A8000088AE00E482A90000A8AF00E4C2A800F4
:187D600000A8AE00E4C2A90000002000C209BD007A003A0000C8AF0093
:187D7800CD02A80000C8AE00CD02A90000E8AF00CD22A80000E8AE00CA
:187D9000CD22A9000108AF00CD42A8000108AE00CD42A9000128AF008D
:187DA800CD62A8000128AE00CD62A90000C0B300DE49B50030003A0084
:187DC0000148AF00E4A2A8000148AE00E4A2A9000168AF00E4E2A800D9
:187DD8000168AE00E4E2A9000188AF00F4C2A8000188AE00F4C2A900E1
:187DF00001A8AF00F4E2A80001A8AE00F4E2A90001C8AF00F502A800B8
:187E080001C8AE00F502A90001E8AF00F522A80001E8AE00F522A9009D
:187E20000208AF00CD82A8000208AE00CD82A9000228AF00CDA2A800FA
:187E38000228AE00CDA2A9000248AF00F442A8000248AE00F442A90094
:187E50000268AF00F462A8000268AE00F462A9000288AF00ECC2A8005D
:187E68000288AE00ECC2A90002A8AF00DC82A80002A8AE00DC82A900B5
:187E800010C0B300DE49B50020003A000148AF00E4A2A8000148AE0014
:187E9800E4A2A9000168AF00E4E2A8000168AE00E4E2A9000188AF005F
:187EB000F4C2A8000188AE00F4C2A90001A8AF00F4E2A80001A8AE0099
:187EC800F4E2A90001C8AF00F442A80001C8AE00F442A90001E8AF00DF
:187EE000F462A80001E8AE00F462A9000208AF00ECC2A8000208AE002F
:187EF800ECC2A9000228AF00DC82A8000228AE00DC82A90020C0B300CA
:187F1000DE49B50010003A000148AF00F442A8000148AE00F442A90087
:187F28000168AF00F462A8000168AE00F462A9000188AF00ECC2A80087
:187F40000188AE00ECC2A90001A8AF00DC82A80001A8AE00DC82A900DF
:187F58003900370000C0B300DE49B50020003A0000C8AF00E4A2A80053
:187F700000C8AE00E4A2A90000E8AF00E4E2A80000E8AE00E4E2A9004A
:187F88000108AF00F4C2A8000108AE00F4C2A9000128AF00F4E2A8005F
:187FA0000128AE00F4E2A9000148AF00F502A8000148AE00F502A90045
:187FB8000168AF00F522A8000168AE00F522A9000188AF00CD82A800D4
:187FD0000188AE00CD82A90001A8AF00CDA2A80001A8AE00CDA2A9008C
:187FE80010C0B300DE49B50010003A0000C8AF00E4A2A80000C8AE00BD
:18800000E4A2A90000E8AF00E4E2A80000E8AE00E4E2A9000108AF0077
:18801800F4C2A8000108AE00F4C2A9000128AF00F4E2A8000128AE00AF
:18803000F4E2A90020C0B300DE49B50000003A00C689BF00CEA4B700D9
:1880480094C8BF00020032000E0007009468EF0095C8BF000200320081
:188060000A0007009568EF0096C8BF0002003200060007009668EF00C0
:1880780097C8BF0002003200020007009768EF000000060006E8B700FC
:1880900000C0B3007A4AB5008F023A0006C8BF008C02320000C2B3005F
:1880A8000648B50091003900F0C7B3000648B50058003A0000012000D3
:1880C00006A8B700BD69EF0006C8BF00BCE9B7000536AF00080037001C
:1880D800000021000016B4000CA0B700BC89BF000003980004B6EC00FD
:1880F00000B6EC000156A900BA69ED00F0CFB300BA49B50027003A003B
:188108007CCABF00BAE9B700BA69ED00BB69ED00F0CFB300BB49B500B4
:1881200003003A007DCABF00BBE9B700BB69ED00BBC9BF00BCE9B700F9
:18813800BD69EF00BC89BF007CCABF000160EF00BC09BC000480BF00FD
:18815000BA49B4000000B400BCA9B70080CB2C00BC09B4000000900010
:18816800BCA9B700BCE9A800BD69EF00BCC9BF00BCE9B7000536AF00F7
:1881800008003700000021000016B4000CA0B700BC89BF0000039800BB
:1881980004B6EC0000B6EC000156A900BBC9BF00BCE9B700BD69EF00D3
:1881B000BC89BF007CCABF000160EF00BC09BC000480BF00BA49B400E3
:1881C8000000B400BCA9B70080CB2C00BC09B40000009000BCA9B70033
:1881E000BCE9A800BD69EF00BCC9BF00BCE9B7000536AF00080037005C
:1881F800000021000016B4000CA0B700BC89BF000003980004B6EC00DC
:1882100000B6EC000156A9003500370010002000BDE9B70006C8BF002E
:18822800BCE9B7000536AF0008003700000021000016B4000CA0B7006B
:18824000BC89BF000003980004B6EC0000B6EC000156A900BA69EC0030
:188258007CCABF00BA49B50023003900BA69EF00BB69EC007DCABF00CD
:18827000BB49B50001003900BB69EF00BBC9BF00BCE9B700BD69EF003C
:18828800BC89BF007CCABF000160EF00BC09BC000480BF00BA49B4000A
:1882A0000000B400BCA9B70080CB2C00BC09B40000009000BCA9B7005A
:1882B800BCE9A800BD69EF00BCC9BF00BCE9B7000536AF000800370083
:1882D000000021000016B4000CA0B700BC89BF000003980004B6EC0003
:1882E80000B6EC000156A900F801370080C0B3000648B50058003A0024
:188300000001200006A8B700BD69EF0006C8BF00BCE9B7000536AF00F7
:1883180008003700000021000016B4000CA0B700BC89BF000003980021
:1883300004B6EC0000B6EC000156A900BA69ED00F0CFB300BA49B500B3
:1883480027003A007CCABF00BAE9B700BA69ED00BB69ED00F0CFB300CA
:18836000BB49B50003003A007DCABF00BBE9B700BB69ED00BBC9BF005A
:18837800BCE9B700BD69EF00BC89BF007CCABF000160EF00BC09BC00A2
:188390000480BF00BA49B4000000B400BCA9B70080CB2C00BC09B4001B
:1883A80000009000BCA9B700BCE9A800BD69EF00BCC9BF00BCE9B7000F
:1883C0000536AF0008003700000021000016B4000CA0B700BC89BF002A
:1883D8000003980004B6EC0000B6EC000156A900BBC9BF00BCE9B7000B
:1883F000BD69EF00BC89BF007CCABF000160EF00BC09BC000480BF0043
:18840800BA49B4000000B400BCA9B70080CB2C00BC09B4000000900055
:18842000BCA9B700BCE9A800BD69EF00BCC9BF00BCE9B7000536AF003C
:1884380008003700000021000016B4000CA0B700BC89BF000003980000
:1884500004B6EC0000B6EC000156A9009D013700A0C0B3000648B500E1
:1884680040003A00BB69EC007DCABF00BB49B50001003900BB69EF0066
:18848000BBC9BF00BCE9B700BD69EF00BC89BF007CCABF000160EF00D7
:18849800BC09BC000480BF00BA49B4000000B400BCA9B70080CB2C000A
:1884B000BC09B40000009000BCA9B700BCE9A800BD69EF00BCC9BF00E9
:1884C800BCE9B7000536AF0008003700000021000016B4000CA0B700C9
:1884E000BC89BF000003980004B6EC0000B6EC000156A900BBC9BF005A
:1884F800BCE9B700BD69EF00BC89BF007CCABF000160EF00BC09BC0021
:188510000480BF00BA49B4000000B400BCA9B70080CB2C00BC09B40099
:1885280000009000BCA9B700BCE9A800BD69EF00BCC9BF00BCE9B7008D
:188540000536AF0008003700000021000016B4000CA0B700BC89BF00A8
:188558000003980004B6EC0000B6EC000156A9005A013700B0C0B30073
:188570000648B50042003A00BB69ED00F0CFB300BB49B50003003A00FB
:188588007DCABF00BBE9B700BB69ED00BBC9BF00BCE9B700BD69EF00B5
:1885A000BC89BF007CCABF000160EF00BC09BC000480BF00BA49B400EF
:1885B8000000B400BCA9B70080CB2C00BC09B40000009000BCA9B7003F
:1885D000BCE9A800BD69EF00BCC9BF00BCE9B7000536AF000800370068
:1885E800000021000016B4000CA0B700BC89BF000003980004B6EC00E8
:1886000000B6EC000156A900BBC9BF00BCE9B700BD69EF00BC89BF0008
:188618007CCABF000160EF00BC09BC000480BF00BA49B4000000B400C6
:18863000BCA9B70080CB2C00BC09B40000009000BCA9B700BCE9A8002D
:18864800BD69EF00BCC9BF00BCE9B7000536AF0008003700000021001B
:188660000016B4000CA0B700BC89BF000003980004B6EC0000B6EC00EE
:188678000156A90015013700C0C0B3000648B50054003A004001200078
:1886900006A8B700BD69EF0006C8BF00BCE9B7000536AF000800370046
:1886A800000021000016B4000CA0B700BC89BF000003980004B6EC0027
:1886C00000B6EC000156A900BA69EC007CCABF00BA49B50023003900D8
:1886D800BA69EF00BB69EC007DCABF00BB49B50001003900BB69EF005C
:1886F000BBC9BF00BCE9B700BD69EF00BC89BF007CCABF000160EF0065
:18870800BC09BC000480BF00BA49B4000000B400BCA9B70080CB2C0097
:18872000BC09B40000009000BCA9B700BCE9A800BD69EF00BCC9BF0076
:18873800BCE9B7000536AF0008003700000021000016B4000CA0B70056
:18875000BC89BF000003980004B6EC0000B6EC000156A900BBC9BF00E7
:18876800BCE9B700BD69EF00BC89BF007CCABF000160EF00BC09BC00AE
:188780000480BF00BA49B4000000B400BCA9B70080CB2C00BC09B40027
:1887980000009000BCA9B700BCE9A800BD69EF00BCC9BF00BCE9B7001B
:1887B0000536AF0008003700000021000016B4000CA0B700BC89BF0036
:1887C8000003980004B6EC0000B6EC000156A900BE003700D0C0B3007E
:1887E0000648B5001F003A00BA69EF00BBC9BF00BCE9B700BD69EF005F
:1887F800BC89BF007CCABF000160EF00BC09BC000480BF00BA49B40095
:188810000000B400BCA9B70080CB2C00BC09B40000009000BCA9B700E4
:18882800BCE9A800BD69EF00BCC9BF00BCE9B7000536AF00080037000D
:18884000000021000016B4000CA0B700BC89BF000003980004B6EC008D
:1888580000B6EC000156A9009C00370010C1B3000648B5000D003A00C5
:18887000C0002000BCA9B7000536AF0008003700000021000016B400E0
:188888000CA0B700BC89BF000003980004B6EC0000B6EC000156A9008E
:1888A0008C00370020C1B3000648B5000D003A00D0002000BCA9B70013
:1888B8000536AF0008003700000021000016B4000CA0B700BC89BF002D
:1888D0000003980004B6EC0000B6EC000156A9007C00370030C1B30056
:1888E8000648B5000D003A00E0002000BCA9B7000536AF0008003700E9
:18890000000021000016B4000CA0B700BC89BF000003980004B6EC00CC
:1889180000B6EC000156A9006C00370040C1B3000648B5000D003A0004
:18893000F0002000BCA9B7000536AF0008003700000021000016B400EF
:188948000CA0B700BC89BF000003980004B6EC0000B6EC000156A900CD
:188960005C00370080C1B3000648B5002F003A007C8ABF00BA09BD00C7
:1889780080EAB70000122000BCA9B7000536AF0008003700000021002E
:188990000016B4000CA0B700BC89BF000003980004B6EC0000B6EC00BB
:1889A8000156A900806AED00F2FF3A00BBC9BF00BCE9B700BD69EF0001
:1889C000BC89BF007CCABF000160EF00BC09BC000480BF00BA49B400CB
:1889D8000000B400BCA9B70080CB2C00BC09B40000009000BCA9B7001B
:1889F000BCE9A800BD69EF00BCC9BF00BCE9B7000536AF000800370044
:188A0800000021000016B4000CA0B700BC89BF000003980004B6EC00C3
:188A200000B6EC000156A9002A003700A0C1B3000648B5000F003A00DB
:188A380010002800BCA9B7000536AF0008003700000021000016B400BE
:188A50000CA0B700BC89BF000003980004B6EC0000B6EC000156A900C4
:188A6800BA69EF00BB69EF0018003700B0C1B3000648B50003003A001E
:188A8000100020007AEAB70012003700E0C1B3000648B5000F003A00AA
:188A980020002800BCA9B7000536AF0008003700000021000016B4004E
:188AB0000CA0B700BC89BF000003980004B6EC0000B6EC000156A90064
:188AC800BA69EF00BB69EF00000037007200370050C0B3007A4AB50055
:188AE0000E003A000768EF0000C2B3000648B5000800390000CAB300A2
:188AF8000648B50005003100F00920000608BD004900DD00CEA4B700FA
:188B1000C6A9B700000020007AEAB70040C0B3007A4AB50010003A0076
:188B280000082000BDE9B70006C8BF00BCE9B7000536AF00080037009E
:188B4000000021000016B4000CA0B700BC89BF000003980004B6EC008A
:188B580000B6EC000156A900000020007AEAB70030C0B3007A4AB5000C
:188B700028003A0000FE2F000648B40006E8B7007CCABF000648B500AF
:188B88000300310006C8BF00BAE9B70000003700000020007AEAB70048
:188BA000BBC9BF00BCE9B700BD69EF00BC89BF007CCABF000160EF00B0
:188BB800BC09BC000480BF00BA49B4000000B400BCA9B70080CB2C00E3
:188BD000BC09B40000009000BCA9B700BCE9A800BD69EF00BCC9BF00C2
:188BE800BCE9B7000536AF0008003700000021000016B4000CA0B700A2
:188C0000BC89BF000003980004B6EC0000B6EC000156A90020C0B300E2
:188C18007A4AB5000B003A0000FE2F000648B40006E8B7007DCABF00AC
:188C30000648B5000300310006C8BF00BBE9B700000037003000200086
:188C48007AEAB70010C0B3007A4AB50012003A00D0C3B3000648B50068
:188C600003003A00200020007AEAB7000C003700C0C4B3000648B500E7
:188C780003003A00400020007AEAB7000600370030C4B3000648B50045
:188C900003003A00500020007AEAB700000037000668EF00000006006A
:188CA8000000000001000000FFFF000000000000000000000000FF00B6
:188CC0000000FF000000000000000000000000000000FF00000000009E
:188CD8000000000000000000000000000000000000000000FFFF000086
:188CF0000100000000000000000000000000FF000000FF00000000006D
:188D0800000000000000FF000000FF0000000000000000000000000055
:188D20000000000000000000000000000100000000000000000000003A
:188D3800FFFF00000000FF000000000000000000000000000000FF0027
:188D50000000FF00FFFF0000000000000000000001000000000000000D
:188D680000000000FFFF00000000000000000000010000000000FF00F5
:188D80000000000000000000000000000000FF000000FF0001000000DC
:188D98000000000000000000FFFF0000000000000000000001000000C4
:188DB000FFFF000000000000FFFF00000000FF000000FF0001000000B0
:188DC800010000000000FF000000FF00FFFF000000000000FFFF000098
:188DE000010000000000000000000000FFFF000001000000000000007B
:188DF800010000000000FF000000FF00FFFF0000FFFF00000000FF0069
:188E10000000FF00010000000000000001000000FFFF0000000000004B
:188E28000100000001000000010000000100000001000000010000002C
:188E400001000000010000000100000001000000010000000100000014
:188E580001000000010000000100000001000000FFFF0000FFFF000002
:188E7000FFFF0000FFFF0000FFFF0000FFFF0000FFFF0000FFFF0000F6
:188E8800FFFF0000FFFF0000FFFF0000FFFF0000FFFF0000FFFF0000DE
:188EA000FFFF0000FFFF000000000000010000000000000000000000BD
:188EB80000000000FFFF000000000000000000000000000001000000A3
:188ED000000000000000000000000000FFFF000000000000000000008C
:188EE80000000000000000000100000000000000000000000000000071
:188F0000FFFF000000000000000000000000000001000000000000005A
:188F18000000000000000000FFFF00000000000000000000FFFF000045
:188F300000000000000000000000000001000000010000000000000027
:188F480000000000FFFF00000000000000000000000000000100000012
:188F600000000000000000000000000000000000FFFF000000000000FB
:188F7800000000000000000001000000000000000000000000000000E0
:188F9000FFFF00000000000000000000000000000100000000000000CA
:188FA80000000000010000000000000000000000FFFF000000000000B2
:188FC000FFFF0000FFFF0000000000000100000000000000000000009C
:188FD80000000000010000000000000000000000000000000000000080
:188FF00001000000000000000000000000000000010000000000000067
:18900800FFFF0000FFFF000000000000FFFF0000000000000000000056
:18902000010000000000000000000000FFFF0000000000000000000039
:189038000100000000000000010000000100000000000000FFFF00001F
:18905000000000000000000000000000FFFF000000000000000000000A
:189068000000000000000000FFFF0000000000000000000000000000F2
:18908000FFFF00000000000001000000010000000000000001000000D7
:189098000000000000000000FFFF0000000000000000000000000000C2
:1890B000000000000000000000000000010000000000000000000000A7
:1890C8000000000000000000000000000000000000000000010000008F
:1890E00000000000000000000000000000000000000000000000000078
:1890F8000000000000000000010000000000000000000000000000005F
:1891100000000000000000000000000000000000010000000000000046
:189128000000000001000000000000000000000000000000000000002E
:1891400000000000000000000000000001000000000000000000000016
:18915800000000000000000000000000000000000000000000000000FF
:18917000010000000000000000000000000000000000000000000000E6
:18918800000000000000000001000000000000000000000000000000CE
:1891A000000000000000000000000000000000000000000000000000B7
:1891B8000000000001000000000000000100000000000000000000009D
:1891D00000000000000000000000000000000000000000000000000087
:1891E8000000000000000000000000000000000000000000000000006F
:1892000000000000000000000000000001000000000000000100000054
:189218000000000000000000000000000000000000000000000000003E
:1892300000000000000000000100000000000000010000000000000024
:189248000000000000000000000000000000000000000000000000000E
:18926000000000000000000000000000000000000000000000000000F6
:18927800000000000000000000000000000000000100000000000000DD
:18929000010000000000000000000000000000000000000000000000C5
:1892A8000000000001000000020000000300000004000000050000009F
:1892C000060000000700000008000000090000000A0000000B00000063
:1892D8000C0000000D0000000E0000000F000000100000001100000027
:1892F000120000001300000014000000150000001600000017000000EB
:1893080018000000190000001A0000001B0000001C0000001D000000AE
:189320001E0000001F0000002000000021000000220000002300000072
:1893380024000000250000002600000027000000000000000100000086
:18935000020000000300000004000000050000000600000007000000EA
:1893680008000000090000000A0000000B0000000C0000000D000000AE
:189380000E0000000F0000001000000011000000120000001300000072
:1893980014000000150000001600000017000000180000001900000036
:1893B0001A0000001B0000001C0000001D0000001E0000001F000000FA
:1893C800200000002100000022000000230000002400000025000000BE
:1893E00026000000270000004000000041000000420000004300000022
:1893F800440000004500000046000000470000004800000049000000B6
:189410004A0000004B0000004C0000004D0000004E0000004F00000079
:189428005000000051000000520000005300000054000000550000003D
:18944000560000005700000058000000590000005A0000005B00000001
:189458005C0000005D0000005E0000005F0000006000000061000000C5
:1894700062000000630000006400000065000000660000006700000089
:18948800000000000100000002000000030000000400000005000000BD
:1894A000060000000700000040000000410000004200000043000000A1
:1894B80044000000450000004600000047000000000000000100000085
:1894D00002000000030000000400000005000000060000000700000069
:1894E80008000000090000000A0000000B0000000C0000000D0000002D
:189500000E0000000F00000010000000110000001200000013000000F0
:18951800140000001500000016000000170000001800000019000000B4
:189530001A0000001B0000001C0000001D0000001E0000001F00000078
:189548002000000021000000220000002300000024000000250000003C
:18956000260000002700000040000000410000004200000043000000A0
:1895780044000000450000004600000047000000480000004900000034
:189590004A0000004B0000004C0000004D0000004E0000004F000000F8
:1895A800500000005100000052000000530000005400000055000000BC
:1895C000560000005700000058000000590000005A0000005B00000080
:1895D8005C0000005D0000005E0000005F000000600000006100000044
:1895F00062000000630000006400000065000000660000006700000008
:189608000000000001000000020000000300000004000000050000003B
:18962000060000000700000008000000090000000A0000000B000000FF
:189638000C0000000D0000000E0000000F0000001000000011000000C3
:1896500012000000130000001400000040000000410000004200000006
:1896680043000000440000004500000046000000470000004800000049
:18968000490000004A0000004B0000004C0000004D0000004E0000000D
:189698004F0000005000000051000000520000005300000054000000D1
:1896B00000000000010000000200000003000000040000000500000093
:1896C800060000000700000008000000090000000A0000000B00000057
:1896E0000C0000000D0000000E0000000F00000010000000110000001B
:1896F800120000001300000014000000150000001600000017000000DF
:18971000400000004100000042000000430000004400000045000000B2
:18972800460000004700000048000000490000004A0000004B00000076
:189740004C0000004D0000004E0000004F00000050000000510000003A
:18975800520000005300000054000000550000005600000057000000FE
:18977000000000000100000002000000030000000400000005000000D2
:18978800060000000700000008000000090000000A0000000B00000096
:1897A0000C0000000D0000000E0000000F00000010000000110000005A
:1897B8001200000013000000140000001500000016000000170000001E
:1897D00018000000190000001A0000001B0000001C0000001D000000E2
:1897E8001E0000001F0000004000000041000000420000004300000026
:18980000440000004500000046000000470000004800000049000000A9
:189818004A0000004B0000004C0000004D0000004E0000004F0000006D
:1898300050000000510000005200000053000000540000005500000031
:18984800560000005700000058000000590000005A0000005B000000F5
:189860005C0000005D0000005E0000005F000000000000000100000079
:18987800020000000300000004000000050000000600000007000000BD
:1898900008000000090000000A0000000B0000000C0000000D00000081
:1898A8000E0000000F0000004000000041000000420000004300000085
:1898C000440000004500000046000000470000004800000049000000E9
:1898D8004A0000004B0000004C0000004D0000004E0000004F000000AD
:1898F000100000001100000012000000130000001400000015000000F1
:18990800160000001700000018000000190000001A0000001B000000B4
:189920001C0000001D0000001E0000001F000000500000005100000018
:189938005200000053000000540000005500000056000000570000001C
:1899500058000000590000005A0000005B0000005C0000005D000000E0
:189968005E0000005F0000000000000001000000020000000300000024
:18998000040000000500000006000000070000000800000009000000A8
:189998000A0000000B0000000C0000000D0000000E0000000F0000006C
:1899B000100000001100000012000000130000004000000041000000D8
:1899C800420000004300000044000000450000004600000047000000EC
:1899E00048000000490000004A0000004B0000004C0000004D000000B0
:1899F8004E0000004F0000005000000051000000520000005300000074
:189A1000140000001500000016000000170000001800000019000000B7
:189A28001A0000001B0000001C0000001D0000001E0000001F0000007B
:189A40002000000021000000220000002300000024000000250000003F
:189A580026000000270000005400000055000000560000005700000053
:189A700058000000590000005A0000005B0000005C0000005D000000BF
:189A88005E0000005F0000006000000061000000620000006300000083
:189AA000640000006500000066000000670000008060A9000040060049
:189AB80000000000000000000000000000000000000000000000000096
:189AD0000000000000000000000000000000000000000000000000007E
:189AE80000000000000000000000000000000000000000000000000066
:189B00000000000000000000000000000000000000000000000000004D
:18A5F80000000000000000007FD637007EDE3700CEE53700D7E537004F
:18A61000E0E53700EBE53700F7E5370001E637000DE6370016E63700A1
:18A628001EE637001DE637001CE637001BE637001AE6370019E63700C7
:18A6400018E63700DBEE370016E6370015E6370014E63700B5EE37005D
:18A6580012E6370011E6370010E637000FE637000EE637000DE63700DF
:18A670000CE637000BE637000AE6370009E6370008E6370007E63700EB
:18A6880006E6370005E6370004E63700CEEE3700D1EE370001E637004D
:18A6A00000E63700FFE53700FEE53700FDE53700FCE53700FBE5370008
:18A6B800FAE53700F9E53700F8E53700F7E53700F6E53700F5E5370015
:18A6D000F4E53700F3E53700F2E53700F1E53700F0E53700EFE5370021
:18A6E800EEE53700EDE53700ECE53700EBE53700EAE53700E9E537002D
:18A70000E8E53700E7E53700E6E53700E5E53700E4E53700E3E5370038
:18A71800E2E53700E1E53700E0E53700DFE53700DEE537009DEE37007B
:18A73000DCE53700DBE53700DAE53700D9E53700D8E53700D7E5370050
:18A74800D6E53700D5E53700D4E53700D3E53700D2E53700D1E537005C
:18A76000D0E53700CFE53700CEE53700CDE53700CCE53700CBE5370068
:18A77800CAE53700C9E53700C8E53700C7E53700C6E53700C5E5370074
:18A79000C4E53700C3E53700C2E53700C1E53700C0E53700BFE5370080
:18A7A800BEE53700BDE53700BCE53700BBE53700BAE53700B9E537008C
:18A7C000B8E53700B7E53700B6E53700B5E53700B4E53700B3E5370098
:18A7D800B2E53700B1E53700B0E53700AFE53700AEE53700ADE53700A4
:10A7F000ACE53700ABE53700AAE53700A9E537003F
:00000001FF
:18000000D9043700B40900003C0C0000500C0000640C00007C0C00007B
:18001800960C0000AC0C0000C60C0000DA0C0000EC0C0000EC0C0000CE
:18003000EC0C0000EC0C0000EC0C0000EC0C0000EC0C0000100E0000C2
:18004800EC0C0000EC0C0000EC0C0000D40D0000EC0C0000EC0C0000E7
:18006000EC0C0000EC0C0000EC0C0000EC0C0000EC0C0000EC0C0000B8
:18007800EC0C0000EC0C0000EC0C0000EC0C0000EC0C0000EC0C0000A0
:18009000EC0C0000EC0C0000EC0C0000EC0C0000EC0C0000EC0C000088
:1800A800EC0C0000EC0C0000EC0C0000EC0C0000EC0C0000EC0C000070
:1800C000EC0C0000EC0C0000EC0C0000EC0C0000EC0C0000EC0C000058
:1800D800EC0C0000EC0C0000EC0C0000EC0C0000EC0C0000EC0C000040
:1800F000EC0C0000EC0C0000EC0C0000EC0C0000EC0C0000EC0C000028
:18010800EC0C0000EC0C0000EC0C0000EC0C0000EC0C0000EC0C00000F
:18012000EC0C0000EC0C0000EC0C0000EC0C0000EC0C0000EC0C0000F7
:18013800EC0C0000EC0C0000EC0C0000EC0C0000EC0C0000EC0C0000DF
:18015000EC0C0000EC0C0000EC0C0000EC0C0000EC0C0000EC0C0000C7
:18016800EC0C0000EC0C0000EC0C0000EC0C0000EC0C0000EC0C0000AF
:18018000EC0C0000EC0C0000EC0C0000EC0C0000EC0C0000EC0C000097
:18019800EC0C0000EC0C0000EC0C0000EC0C0000EC0C0000EC0C00007F
:1801B000EC0C0000EC0C0000EC0C0000EC0C0000EC0C0000EC0C000067
:1801C800EC0C0000EC0C0000EC0C0000EC0C0000EC0C0000EC0C00004F
:1801E000EC0C0000EC0C0000EC0C0000EC0C0000EC0C0000EC0C000037
:1801F800EC0C0000EC0C000000530000025300000453000006530000A7
:18021000085300000A5300000C5300000E530000105300001253000096
:180228001453000016530000185300001A5300001C5300001E53000036
:1802400020530000225300002453000026530000285300002A530000D6
:180258002C5300002E5300003053000032530000345300003653000076
:18027000385300003A5300003C5300003E530000405300004253000016
:180288004453000046530000485300004A5300004C5300004E530000B6
:1802A00050530000525300005453000056530000585300005A53000056
:1802B8005C5300005E53000060530000625300006453000066530000F6
:1802D000685300006A5300006C5300006E530000705300007253000096
:1802E8007453000076530000785300007A5300007C5300007E53000036
:1803000080530000825300008453000086530000885300008A530000D5
:180318008C5300008E5300009053000092530000945300009653000075
:18033000985300009A5300009C5300009E530000A0530000A253000015
:18034800A4530000A6530000A8530000AA530000AC530000AE530000B5
:18036000B0530000B2530000B4530000B6530000B8530000BA53000055
:18037800BC530000BE530000C0530000C2530000C4530000C6530000F5
:18039000C8530000CA530000CC530000CE530000D0530000D253000095
:1803A800D4530000D6530000D8530000DA530000DC530000DE53000035
:1803C000E0530000E2530000E4530000E6530000E8530000EA530000D5
:1803D800EC530000EE530000F0530000F2530000F4530000F653000075
:1803F000F8530000FA530000FC530000FE53000000C0B300ECEAB700BD
:1804080060EDB70061EDB7006AEDB70066EDB700CCEAB700FAEAB700B3
:1804200010002000F9EAB70020002000F8EAB70030002000F7EAB70039
:1804380040002000F5EAB70080002000F4EAB700F0CFB300F3EAB7007B
:18045000F00F20006BEDB700800F2000F2EAB70010002000F1EAB70062
:18046800B0002000F0EAB700000C2000D3EAB70080002000DDEAB7005D
:18048000B0002000DCEAB70000002000E4EAB70000002000E5EAB700CC
:1804980000002000E0EAB70000002000E1EAB700C0FE2000EAAAB700E0
:1804B0002882BF000020EC002062AF00020037004100DD0001003700FF
:1804C8004200DD0064AAB7000020EF006BCDBF00BA0AB400640ABC0090
:1804E0000680BF0003003A000480BF000CA1B700010037000CA1EF0007
:1804F800EC02A900803E20002AAAB7002C2AEC0061CDBF0002003A0081
:18051000EC02A90001003700EC22A90000E0200014A0B700CB6AEF00BE
:180528008C6AEF00E96AEF006D050700ECCABF0088EAB70000CCB300FE
:18054000EC4AB600F8FF3200CBEAEF00F0C1B300884AB600D2EAB7008B
:1805580000CCB300884AB600D3EAB70000CCB300D34AB50004003A0081
:18057000F0CFB300884AB50001003A00E7FF370000C8B300D34AB500D5
:1805880016003A00F0C3B300884AB600D1EAB700E9EAEF00D1CABF008F
:1805A0004200A90000C0D60000C0D60000C0D60000C0D60017E0B70052
:1805B80000C0D700F24AB60016E0B70017C0BF00F14AB600F04AB40080
:1805D00017E0B700C4E9EF003B40780088EAB7000000370088CABF0065
:1805E800005D780000CCB300884AB600D3EAB700F0C3B300884AB600BD
:18060000D1EAB70080C0B300884AB600CEEAB70040C0B300884AB6004B
:18061800EEEAB70030C0B300884AB600EDEAB70000C2B300884AB60085
:18063000EFEAB70000CCB300D34AB5000A003A0000C2B300EF4AB5002A
:1806480007003A0000C0B300E94AB500030032000B409000005D780019
:18066000010037004C05070000C4B300D34AB50065003A0040C0B30057
:18067800EE4AB5000A003A0000C0B300E94AB500050032003B407800B4
:18069000005D78003B407800005D7800020037003D0507003C050700EB
:1806A80000C2B300EF4AB50055003A0000C0B300ED4AB5000A003A00A5
:1806C00000C1B300884AB6000600320000C0B300E94AB500020032005F
:1806D8003B407800005D7800010037002C05070010C0B300ED4AB50063
:1806F0000D003A0000C1B300884AB6000800320000C0B300E94AB5001A
:18070800040032003B407800005D78003B407800005D780002003700DA
:180720001D0507001C05070020C0B300ED4AB50013003A0000C1B30030
:18073800884AB6000C00320000C0B300E94AB500080032003B4078005B
:18075000005D78003B407800005D78003B407800005D78003B40780039
:18076800005D780004003700090507000805070007050700060507001B
:1807800030C0B300ED4AB5001F003A0000C1B300884AB6001400320037
:1807980000C0B300E94AB500100032003B407800005D78003B407800F1
:1807B000005D78003B407800005D78003B407800005D78003B407800D9
:1807C800005D78003B407800005D78003B407800005D78003B407800C1
:1807E000005D780008003700EB040700EA040700E9040700E80407001B
:1807F800E7040700E6040700E5040700E404070000C0B300E94AB500CC
:1808100002003A0000C0B30088EAB70000C0B3000045980000C0B30035
:18082800E94AB5000A0032003B40780088EAB700005D780014C0BF0010
:18084000EA4AB50015C0BF00EBCAB5000200310000C1B300616DB7008D
:1808580088CABF0063FF3A00E96AEF0000C0B3000045980062CDBF005B
:18087000090032008CCABF007F040700ECCABF008C4AB5000400320060
:1808880010C0B300616DB700636DEC0021FF3700CB6AEF0000E0200019
:1808A00014A0B7008B6AEF003A40780088EAB70000CCB300884AB600CF
:1808B800D3EAB70080C0B300884AB600CEEAB70040C0B300884AB6008F
:1808D000EEEAB70030C0B300884AB600EDEAB70000C2B300884AB600CB
:1808E800EFEAB70000CCB300D34AB500BF003A00F0C1B300884AB60032
:18090000D2EAB70000C2B300884AB600EFEAB70016C0BF00E2EAB700C7
:1809180017C0BF00E3EAB70000C1B300D24AB5001100310000D6200030
:1809300016A0B70016C0BF00D24AB40016E0B70017C0BF00FACAB40022
:1809480017E0B70000C2B300EF4AB50003003A003A40780080459800FA
:18096000020037000B409000810407009D00370000C2B300EF4AB500A8
:1809780042003A0070CFB300884AB50002003A003A4078003C003700D1
:1809900080CFB300884AB50009003A0000C0B3006A4DB50003003A0067
:1809A8003A407800E4EAB700020037003A407800E0EAB70030003700AD
:1809C00090CFB300884AB50009003A0000C0B3006A4DB50003003A0027
:1809D8003A407800E5EAB700020037003A407800E1EAB7002400370087
:1809F000A0CFB300884AB50011003A0000C0B3006A4DB50007003A00DB
:180A08003A407800E44AB400E4EAB700E5CABF00FACAB400E5EAB70011
:180A2000060037003A407800E04AB400E0EAB700E1CABF00FACAB4004E
:180A3800E1EAB70010003700D0CFB300884AB50003003A003A407800D5
:180A5000CCEAB7000A003700E0CFB300884AB50007003A003A407800C4
:180A6800ECEAB700A0C5B300EC4AB50001003A003B0237000000370000
:180A80005800370000CDB300884AB50003003A0070C3B3003604070064
:180A98005200370010CDB300884AB50003003A0090C4B3003004070027
:180AB0004C00370020CDB300884AB50003003A0070C3B3002A0407002C
:180AC8004600370030CDB300884AB50003003A0030C3B3002404070050
:180AE0004000370040CDB300884AB50003003A00D0C0B3001E04070097
:180AF8003A00370050CDB300884AB50003003A00E7CABF00180407004E
:180B10003400370060CDB300884AB50003003A00E6CABF001204070032
:180B28002E00370070CDB300884AB50003003A0040C9BF000C040700BD
:180B400028003700A0CDB300884AB50003003A0000C0B30006040700D6
:180B580022003700C0CDB300884AB50003003A0080C0B300000407002A
:180B70001C00370080CDB300884AB50008003A0000C0B3006A4DB50072
:180B880002003A00E4CABF0001003700E0CABF00F503070011003700C4
:180BA00090CDB300884AB50008003A0000C0B3006A4DB50002003A0049
:180BB800E5CABF0001003700E1CABF00EA03070006003700F0CDB30074
:180BD000884AB50003003A00A0C5B300E403070000003700E2CABF00A1
:180BE80016E0B700E3CABF0017E0B700F0C3B300884AB600D1EAB700CE
:180C000000C4B300D34AB500CD013A0040C0B300EE4AB5000C003A00A5
:180C180000C0B3006A4DB50005003A003A407800E4EAB7003A4078003D
:180C3000E5EAB700040037003A407800E0EAB7003A407800E1EAB70004
:180C480000C0B3006A4DB50005003A00E4CABF0016E0B700E5CABF00EE
:180C600017E0B70005003700E0CABF0016E0B700E1CABF00F04AB40024
:180C780017E0B70020C0B3006C4DB50002003A004200A9000600370051
:180C900000C0B3006A4DB50002003A004200A900010037004200A90023
:180CA8000400390000DB200016A0B70000C2B300616DB70010C0B30012
:180CC0006C4DB50016003A003220EF004200F800000E20004200B700BC
:180CD80042A0B70000DB20001AA0B70000402500E44AB40018A0B70049
:180CF00080002000ACAAB7001880BF001040BA00804698001820EC005C
:180D08001A20EC00AC2AED00F9FF3A0000DB200016A0B7004200F90015
:180D200020C0B3006C4DB50034003A0080002000DDEAB700B00020005E
:180D3800DCEAB7004200A900DA8ABF000080D700D6AAB700D88ABF0069
:180D50000080D7000000A900D4AAB700F0FF2700E40AB6004200A900B1
:180D68000080D7000000A900D40AB400D4AAB70000C8B300E54AB6004C
:180D80001B003A0000DB200016A0B70000C2B300EF4AB50015003200F4
:180D98001400F800D68ABF0032A0B700D48ABF0014A0B70000DB20000C
:180DB0001AA0B7001480BF001000BA00801E78001480BF001080BA00EA
:180DC800801E780014A0EC001480BF001000BA00801E78001480BF00D7
:180DE0001080BA00801E78001400F9000300370080AD2000E44AB40025
:180DF80016A0B70000C2B300EF4AB500FA003A0000C0B300ED4AB50080
:180E100004003A003A407800805D7800F9CABF00FE02070010C0B30039
:180E2800ED4AB50007003A000400FC003A407800805D78003A4078004C
:180E4000805D7800F8CABF00F402070020C0B300ED4AB5000B003A0003
:180E58000800FC003A407800805D78003A407800805D78003A407800FE
:180E7000805D78003A407800805D7800F5CABF00E602070030C0B300BE
:180E8800ED4AB50013003A001000FC003A407800805D78003A407800D4
:180EA000805D78003A407800805D78003A407800805D78003A40780065
:180EB800805D78003A407800805D78003A407800805D78003A4078004D
:180ED000805D7800F4CABF00D002070010C0B3006C4DB50052003A00E2
:180EE8003220EF004200F800000E20004200B70042A0B700E5CABF0049
:180F000047003A0000C8B300E44AB60040003A001400F800004025000E
:180F180014A0B70000042000ACAAB7001480BF001000BA00000DBB0040
:180F300000002000008DBB0014A0EC00AC2AED00F8FF3A003220EF006C
:180F48002004240060A7B7000040250014A0B7001000BA00000DBB0029
:180F600040A7A9004200F800000E20004200B70042A0B700500520007A
:180F780066A7B700A00A200066A7B70061E7A80000000000000000001F
:180F90004200F9000060FE0000DB20001AA0B70000402500E40AB4003D
:180FA80014A0B70080002000ACAAB7000D409000004DBB001420EC0014
:180FC0001A20EC00AC2AED00FAFF3A0040A7A9001000240060A7B7007B
:180FD8005005200066A7B700A00A200066A7B70061E7A800000000004A
:180FF0000000000061E7AF00FEFF37000000200060A7B7000060FE0082
:181008001400F9000300370000C2B300616DB7006C6DEF00030037008D
:1810200000C2B300616DB7006C6DEF004200F90020C0B3006C4DB500BA
:181038006C003A0070C7B300DF4AB50014003A004200F800000E20007C
:181050004200B70042A0B7001400F800D68ABF0032A0B700D48ABF0025
:1810680014A0B700000420000AA0B700F0FF2F00000DBB00008DBB0052
:1810800014A0EC000A20ED00FAFF3A001400F900DF6AEF004200F900EE
:18109800D0CFB300DF4AB50017003A004200F800000E20004200B7005E
:1810B00042A0B7001400F80040A7A9001000240060A7B700500520008C
:1810C80066A7B700A00A200066A7B70061E7A8000000000000000000CE
:1810E00061E7AF00FEFF37000000200060A7B7000060FE001400F90084
:1810F800DF6AEF004200F900E0CFB300DF4AB5001D003A004200F8009C
:18111000000E20004200B70042A0B7001400F800D68ABF0032A0B70053
:18112800D48ABF0014A0B700000DBB002004240060A7B70040A7A900C9
:181140004200F800000E20004200B70042A0B7005005200066A7B70064
:18115800A00A200066A7B70061E7A80000000000000000004200F900C6
:181170000060FE001400F900DF6AEF004200F90000C2B300EF4AB50026
:1811880018003A0000C0B300DF4AB50015003A004200F800000E2000F5
:1811A0004200B70042A0B7001400F800D68ABF0032A0B700D48ABF00D4
:1811B80014A0B70000DB20001AA0B7003D007800000DBB003D00780016
:1811D000009DBB003D007800000DBB003D007800009DBB001400F90018
:1811E8004200F9005400370000C0B300ED4AB50007003A000400FC0089
:181200003B407800BDEAB700BDCABF0058020700F9CABF000102070052
:1812180010C0B300ED4AB5000B003A000400FC003B407800BDEAB700B9
:181230003B407800BEEAB700BDCABF004C020700BECABF004A0207001F
:18124800F8CABF00F301070020C0B300ED4AB50013003A000800FC0042
:181260003B407800BDEAB7003B407800BEEAB7003B407800BFEAB70080
:181278003B407800C0EAB700BDCABF003A020700BECABF0038020700F9
:18129000BFCABF0036020700C0CABF0034020700F5CABF00DD010700D6
:1812A80030C0B300ED4AB50023003A001000FC003B407800BDEAB700E5
:1812C0003B407800BEEAB7003B407800BFEAB7003B407800C0EAB7001D
:1812D8003B407800C1EAB7003B407800C2EAB7003B407800C3EAB700FC
:1812F0003B407800C4EAB700BDCABF001C020700BECABF001A020700B9
:18130800BFCABF0018020700C0CABF0016020700C1CABF001402070095
:18132000C2CABF0012020700C3CABF0010020700C4CABF000E02070086
:18133800F4CABF00B70107000A409000FA4AB70057FD3A0062CDBF0010
:18135000020032008BCABF00050207004889BF004CA9B70065FC37005B
:181368000020EF000220EF000420EF000620EF000820EF000A20EF00F5
:181380000C20EF000E20EF001020EF001220EF001420EF001620EF0095
:181398001820EF001A20EF001C20EF0000DC20001EA0B70000E0200051
:1813B00020A0B7000080200014A0B700F07F200002A0B700000020009B
:1813C800004598001420EC000220ED00FBFF3A003220EF004400A800A0
:1813E00083E0A90081E0A9008560A9009560A90000002700A820B7000D
:1813F80000002600A620B700C8A2EF00D0A2EF00E0A2EF00E8A2EF0096
:18141000F0A2EF000078200050A7B7005010210000A3B70001E3A90095
:1814280000F02F0002A3B700101020000AA3B700101020000CA3B700E7
:18144000101020000EA3B7001010200010A3B70001E3A800A0002000F6
:181458009AAAB7006A0107009A2AED00FDFF3A00E66AEF00E60AA90050
:18147000EAC2AF00E60AA800E62AA900F262AF00E62AA800E64AA90024
:18148800F242AF00E64AA80092EAA800E64AAE0003003700E62AAE0097
:1814A0000100370092EAA9000000280020A2B7000040220022A2B70059
:1814B8008540A90042C7A9000000200044A7B700E001200046A7B70095
:1814D0000000280004A1B700F0FF2F0000A1B7000001280010A1B70079
:1814E8000000280012A1B700001920000EA1B7000000280020A1B7001B
:18150000001920001CA1B70000002000CCA2B700F00F2C00C8A2B70095
:1815180000002400D4A2B700F0FB2900D0A2B70000002000DCA2B700D8
:18153000F0FA2F00D8A2B70000002000E4A2B700A0702F00E0A2B70084
:1815480090002000ECA2B70040FB2F00E8A2B70000002000F4A2B7007E
:1815600030C32F00F0A2B700100020009AAAB700250107009A2AED00FF
:18157800FDFF3A002682BF002202AF00F8FF37002682BF002202AF0083
:18159000FDFF3700B42AEF00B22AEF00C86AEF00C76AEF00C66AEF0018
:1815A800B7EAEF00E00020005CA9B700100020004CA9B70010002000D3
:1815C00040A9B700A0002000BAAAB70092EAAE005C003700200020009B
:1815D80008A0B7003220EF00004025000800B4001000BA0008A0B70011
:1815F00008C0BF0062EDB7000000200008A0B7003220EF000040250031
:181608000800B4001000BA0008A0B7000000200028A2B70000C0B300D1
:181620000840B50002003A003010200028A2B70010C0B3000840B50018
:1816380002003A001008200028A2B70020C0B3000840B50002003A00D9
:181650000004200028A2B70030C0B3000840B50002003A00A00220003F
:1816680028A2B70040C0B3000840B50002003A005001200028A2B7000B
:1816800050C0B3000840B50002003A00A000200028A2B70060C0B30042
:181698000840B50003003A005001200028A2B7002062A80070C0B30001
:1816B0000840B50003003A00A000200028A2B7002062A80080C0B3008A
:1816C8000840B50002003A001000200028A2B70090C0B3000840B50020
:1816E00002003A000000200028A2B700A0C0B3000840B50003003A00C8
:1816F8001000200028A2B7002062A800B0C0B3000840B50003003A00A2
:181710000000200028A2B7002062A800400620000AA0B7000521B80051
:181728000680BF0003003A000480BF0048A9B7000100370048A9EF0024
:1817400046003700F00F200062EDB7004000200008A0B7000000200010
:1817580028A2B70000C0B3000840B50002003A003010200028A2B7006B
:1817700010C0B3000840B50002003A001008200028A2B70020C0B30059
:181788000840B50002003A000004200028A2B70030C0B3000840B500CB
:1817A00002003A00A002200028A2B70040C0B3000840B50002003A00C6
:1817B8005001200028A2B70050C0B3000840B50002003A00A00020006B
:1817D00028A2B70060C0B3000840B50003003A005001200028A2B70081
:1817E8002062A80070C0B3000840B50003003A00A000200028A2B70061
:181800002062A80080C0B3000840B50002003A001000200028A2B700C9
:1818180090C0B3000840B50002003A000000200028A2B700A0C0B300C8
:181830000840B50003003A001000200028A2B7002062A800B0C0B30068
:181848000840B50003003A000000200028A2B7002062A8002222A90096
:181860008560A9009560A80092EAAE0001003700E3013700E2FA3700B5
:181878007EA9B7007C09F9007609F9007609F8007C09F80076A9ED0084
:181890007A29EC000010200078A9B700004006007EA9B7007C09F90007
:1818A8007609F9007609F8007C09F80076A9ED007A29EC0010002000F1
:1818C00078A9B700004006007EA9B7007C09F9007609F9007609F800A7
:1818D8007C09F80076A9ED007A29EC002000200078A9B7008060A9003F
:1818F00040A7A800004006007EA9B7007C09F9007609F9007609F800C0
:181908007C09F80076A9ED007A29EC003000200078A9B70000DC20008B
:181920001EA0B7008040A900004006007EA9B7007C09F9007609F900B7
:181938007609F8007C09F80076A9ED007A29EC004000200078A9B700D0
:181950008080A900004006007EA9B7007C09F9007609F9007609F80045
:181968007C09F80076A9ED007A29EC005000200078A9B700E083BF00E5
:181980007CA9B70080A0A900004006007EA9B7007C09F9007609F90090
:181998007609F8007C09F80076A9ED007A29EC00600020007CA9B7004C
:1819B000004006007EA9B7007C09F9007609F9007609F8007C09F80011
:1819C80076A9ED007A29EC00700020007CA9B70000400600D0C0B30077
:1819E00001000700A0C0B3009EEAB7002222A9000060FE002322AF0056
:1819F800FDFF37009ECABF0024E2B700000006001041230090A9B70056
:181A10009029ED00FEFF3A0000000600CDEAB700CECABF004220AE0006
:181A28000700370016C0BF00CD4AB50016E0B70017C0BF00FACAB5004B
:181A400017E0B7000B00370000C0B3006A4DB50005003A0016C0BF00EB
:181A5800E4EAB70017C0BF00E5EAB700030037000020EF00CDCABF0036
:181A7000E02AB40000000600C6CABF0001003A00FDFF370000D72000E6
:181A8800B20AB40018A0B700003020001C00600009003200CBCABF000C
:181AA0000700320000C4B300614DB70061EDB7000500FC0000DC200017
:181AB8001EA0B70097FA37000C409000ECEAB7001820EC000C40900070
:181AD000B8EAB700C66AED00B2AAEC00B2CAA900ECCABF0000000600A0
:181AE800C6CABF0001003A00FDFF370000D72000B20AB40018A0B70053
:181B0000003020001C00600009003200CBCABF000700320000C4B300C2
:181B1800614DB70061EDB7000500FC0000DC20001EA0B7007BFA37002D
:181B30000C409000ECEAB7001820EC000C409000B8EAB700C66AED00BE
:181B4800B2AAEC00B2CAA900ECCABF00ECCABF008CEAB60000F02000F2
:181B60008C4AB4001040BA008CEAB70000000600ECEAB700ECCABF00A4
:181B78009BFF0700ECCABF008BEAB60000F020008B4AB4001040BA0071
:181B90008BEAB70000000600D3FF0700ECCABF00005D780000000600E2
:181BA8008560A9000000F8001000F80026C2BF008AEAB70000042000A1
:181BC000C64AB5001100320000D72000B40AB40010A0B7008ACABF0022
:181BD800004498001020EC0084E0AE000200370010C0B30001003700F7
:181BF00000C0B300004498000621EF0084E0A900C66AEC00B4AAEC0005
:181C0800B4CAA9002202AF00E8FF37001000F9000000F9000040060064
:181C20000000F80094E0A900B7EAEF0011E1A9000621EF000000F9005D
:081C380084E0A9000040060051
:181E0000005E0000BCE20000613F0000DD830000C29C00007E200000D2
:181E1800A3FD00001F4100009DC30000217F0000FCA20000401E0000B6
:181E30005F010000E3BD00003E60000082DC0000237D00009FC100009E
:181E4800421C0000FEA00000E1BF00005D03000080DE00003C6200008A
:181E6000BEE00000025C0000DF810000633D00007C220000C09E000072
:181E78001D430000A1FF000046180000FAA40000277900009BC5000056
:181E900084DA000038660000E5BB000059070000DB850000673900003E
:181EA800BAE400000658000019470000A5FB000078260000C49A00002A
:181EC000653B0000D9870000045A0000B8E60000A7F900001B4500000E
:181ED800C69800007A240000F8A60000441A000099C70000257B0000FA
:181EF0003A64000086D800005B050000E7B900008CD20000306E0000E2
:181F0800EDB30000510F00004E100000F2AC00002F71000093CD0000C5
:181F2000114F0000ADF30000702E0000CC920000D38D00006F310000AD
:181F3800B2EC00000E500000AFF10000134D0000CE900000722C000099
:181F50006D330000D18F00000C520000B0EE0000326C00008ED0000081
:181F6800530D0000EFB10000F0AE00004C12000091CF00002D73000065
:181F8000CA94000076280000ABF500001749000008560000B4EA000051
:181F980069370000D58B000057090000EBB50000366800008AD4000035
:181FB00095CB000029770000F4AA000048160000E9B70000550B00001D
:181FC80088D60000346A00002B75000097C900004A140000F6A8000009
:181FE000742A0000C8960000154B0000A9F70000B6E800000A540000F1
:081FF800D78900006B350000E1
:18A8000009000000FFFF00000100000014040000000000000000000020
:18A8180000000000000000000000000000000000000000000000000028
:18A8300000000000000000000000000000000000000000000000000010
:18A84800000000000000000000000000000000000000000000000000F8
:18A86000000000000000000000000000000000003200000000000000AE
:18A8780000000000000000000000000000800000102700001E000000F3
:18A89000008000006400000000000000000000000000000000000000CC
:18A8A80000000000000000000000000000000000000000000000000098
:18A8C00000000000000000000000000000000000000000000000000080
:18A8D80000000000000000000000000000000000000000000000000068
:10A8F000785600003412000000000000AA55000045
:00000001FF
:0200000401F009
:100000000F000000FF000000070000008300000058
:10001000C50000004000000007000000C300000011
:00000001FF
